:020000022000DC
:1060000000000120756302005D6302005F6302000F
:106010006163020063630200656302000000000028
:1060200000000000000000000000000067630200A4
:1060300069630200000000006B6302006D630200F0
:10604000E98902006F630200BD8B02001596020011
:106050006F6302006F630200718A02006F630200C7
:106060006F6302006F6302003D9B02006F630200DA
:106070006F6302006F6302006F6302006F630200D0
:106080006F630200696F02006F6302006F630200BA
:106090006F6302006F630200FDA202006F630200E3
:1060A0006F6302006F6302006F6302006F630200A0
:1060B0006F6302006F630200000000000000000038
:1060C0006F6302006F6302006F6302006F63020080
:1060D0006F6302006F6302006F6302000000000044
:1060E00000000000000000000000000000000000B0
:1060F00000000000000000000000000000000000A0
:10610000000000000000000000000000000000008F
:10611000000000000000000000000000000000007F
:10612000000000000000000000000000000000006F
:10613000000000000000000000000000000000005F
:10614000000000000000000000000000000000004F
:10615000000000000000000000000000000000003F
:10616000000000000000000000000000000000002F
:10617000000000000000000000000000000000001F
:10618000000000000000000000000000000000000F
:1061900000000000000000000000000000000000FF
:1061A00000000000000000000000000000000000EF
:1061B00000000000000000000000000000000000DF
:1061C00000000000000000000000000000000000CF
:1061D00000000000000000000000000000000000BF
:1061E00000000000000000000000000000000000AF
:1061F000000000000000000000000000000000009F
:10620000354936480A1A02D0072291438D4634494F
:1062100034480A1A06D00722914381F309880222E2
:1062200082F3148830483149314A00F044F831484B
:106230003149324A00F03FF831483249324A00F0E1
:106240003AF832483249334A00F035F83248334997
:10625000334A00F030F833483349344A00F02BF821
:1062600033483449344A00F026F83448344900228F
:1062700000F02CF833483449002200F027F8334866
:106280003349091A082902DB002202604160314AC1
:1062900090471F481F49884205D00268043003B464
:1062A000904703BCF7E700208646EC46002000211B
:1062B000294A9047FEE7884207D0521A05D0037852
:1062C00001300B700131013AF9D17047884202D098
:1062D00002700130FAE770470000012000E0002062
:1062E0000000012000000120E8C60200D82A00209A
:1062F0002C2B0020D0630200D063020028BF0200D4
:10630000E8C60200D82A0020D82A00201CC00200BB
:106310001CC002001CC002001CC002001CC0020005
:106320001CC002001CC002001CC00200E7C6020024
:106330003CC702002C2B00202C2B00202C2B0020F3
:106340005CB000205CB000205CB000205CB000209D
:106350005CD000209D630200359C0200FEE7FEE752
:10636000FEE7FEE7FEE7FEE7FEE7FEE7FEE7FEE705
:1063700000F002B8FFF7FCBF0F484FF00701884359
:1063800085460E4880470E48016841F4700101605F
:10639000BFF34F8FBFF36F8FFFF732BF09480A4932
:1063A0000A4A884207D0521A05D0037801300B7090
:1063B0000131013AF9D1704700000120D184020077
:1063C00088ED00E01CC00200D82A0020D82A002056
:1063D0007047000007B5044B0093044A402300F0C7
:1063E00032F803B05DF804FBF16302002D2B0020AE
:1063F0002DE9F84388461446B2B10F4B0F4E0325E2
:10640000002743F00109224608EB0701002003F0B2
:10641000C1FD0744241A48B933782BB14FF47A40B0
:10642000C847013D02D13570BDE8F88301233370C0
:10643000002CE8D1F8E700BF20C002002C2B002080
:10644000704703F0D7BDF0B595B01D461646084617
:106450000C4601F0E9F81A9B0D93CDE9086500257B
:106460002B46082205A920460A958DF82C500C953C
:1064700001F0F6F8079B0293069B03939DF81430F6
:106480008DF8115003F00302012A1DD1BDF814202C
:10649000059DC3F3C203C2F383168DF81030B2001A
:1064A00008230EA9204601F0DBF8C5F3952508ABBB
:1064B0000093324602AB0EA9284600F03BFB204673
:1064C00001F0B6F815B0F0BD022AF8D1BDF81650AB
:1064D000C3F3C203C5F389158DF810300827082DC2
:1064E0002E4628BF08263B4632460EA9204601F01C
:1064F000B7F8AD1B08AB02AA31460EA8374400F02E
:106500007DFB002DEBD1DAE738B50A4DFFF799FF97
:106510000421284600F078FA074B01245C7100F052
:1065200037FC042105F1100000F06EFA034B5C719A
:1065300038BD00BFFCBF0200D82A0020E02A00209E
:10654000037813F0040216D003F00303012B03D0E9
:10655000022B09D0012070470A6800880232C0F37C
:10656000831002440A60F5E70B684288023303EBAC
:1065700092130B60EEE71046704700002DE9F04FD4
:10658000DFF81CA187B00F4600230446861C0DF1DE
:10659000070015468DF8073000F096FCDAF8042065
:1065A0003A60DAF8083003F580739B1A0AF21C4748
:1065B0000AF583690AF21448B3421AD30020002D69
:1065C00069D004F00F039B0143F0050363F30F0050
:1065D000DAF80430DAB2033233444AF822009DF884
:1065E0000700CAF8043000F093FC012007B0BDE8B2
:1065F000F08F0121384600F046FD484600F05BFD73
:10660000404600F058FDDAF808000290C0B20330AE
:106610000AEB800002A9FFF793FF029B30BBDAB2BE
:106620000AEB8202D16803919A1C0133DBB20AEBB8
:1066300083030292D3F80CB001F00303012B22D0A4
:10664000022B15D08346404600F038FD10B1029B66
:10665000CAF808305946384600F015FDDAF8083017
:10666000DAF8042003F580739B1AA5E7D8B2CEE7C9
:10667000BDF80E30C3F3891303334FEA1B4B02EB13
:1066800093030293DFE7BDF80C30C3F383134FEAA3
:106690001B4B1344F5E7A40544F0060098E700BF40
:1066A000402C0020064B074810B501221A7000F05C
:1066B00074FF044610B9044800F0DCFF204610BD0A
:1066C000402C002060BF02006CC0020030B50A4CB4
:1066D00071B10A4A0A49121BD20800239A4201D119
:1066E000002030BD31F82350854202D00133F5E758
:1066F000034654F83300F4E774BF0200FCBF020005
:10670000D82A0020094B013903EBC000032909D81E
:10671000DFE801F00A0204060420704700797047A0
:1067200040797047002070470220704774BF020014
:10673000034BD3E90130C31A58425841704700BF98
:10674000402C00202DE9F04186B0FFF7F1FF05460F
:10675000002840F0ED80774CC4F81804BFF34F8F49
:10676000A3680293DBB2033304EB830002A9FFF7B3
:10677000E7FE029B18B1D4F81824002A5AD0DAB2E6
:10678000991C013304EB8202DBB204EB8303D26871
:10679000DB68049302F00303022B0392029154D1AD
:1067A000BDF80E306448C3F38917502F3E4628BF0A
:1067B000502606F1080166F38F13C1F30901ADF805
:1067C0000E3000F002FF0546002800F09C8000F02B
:1067D0002BFF0023082203A9284600F037FF029967
:1067E000CB43DBB20133C9B20331B6EB830F4FEABF
:1067F000830204EB810125D95FFA82F80823A6EB16
:106800000806284600F022FFF6B208F108034B49BB
:1068100003F0FC033246284600F018FF029B0337C2
:1068200003EB97070297D4F81834002B43D1D4F820
:10683000106453E062689A4294D8A260284606B079
:10684000BDE8F08108233246E5E7012B5BD1BDF8B6
:106850000C303948C3F38311062928BF062161F3A0
:106860008913023101F00F018900ADF80C3000F0FE
:10687000ACFE0546002846D000F0D6FE00230822D4
:1068800003A9284600F0E2FE0026BDF80C20C2F362
:106890008312B300964203F10803C4D202994A1C42
:1068A000C9B20331029204EB81010422284600F0B0
:1068B000CDFE0136E9E7284600F0BAFEFFF738FFC3
:1068C00080F00100C5B2B9E7F3685B7923B13368A2
:1068D00029461B6830469847F3681E68002EF3D19E
:1068E000284600F0A5FE0DF107008DF8076000F0C6
:1068F000EBFAD4F818340BB9029BA3609DF807009B
:1069000000F006FBDAE7D4F8104454B90C4B0D48FC
:106910000D49C01AC008000440F0020000F05CF805
:10692000CCE7236820469B689847E3681C68ECE73F
:10693000002583E7402C002060BF02004C2C002083
:1069400074BF0200A4BF020055C002002DE9F34746
:1069500004460E46924601A9012218469946FFF7C1
:106960000DFE1B4F10B3019D4FF00008AA1CC84537
:1069700008EB020123D11748002100F055FB80F3FA
:106980001000000440EA1440E4006B1C04F03804DA
:10699000DBB2EDB244F0010407EB8303033544EAB4
:1069A000881444EA8624D86047F825403B781BB118
:1069B000FFF7C8FE0028FBD102B0BDE8F087C9B2DE
:1069C00007EB81015AF82830CB6008F10108CEE7C7
:1069D000402C00205C30002000231A46FFF7B6BF91
:1069E00007B50123019201AAFFF7B0FF03B05DF8DC
:1069F00004FB07B5CDE9002302236A46FFF7A6FF93
:106A000003B05DF804FB000030B50F4CD4F810243F
:106A100003460020114631B9D96808714AB9C4F853
:106A200010340A6030BDC9680D79854206D0096806
:106A3000F1E7D26814680C601360F3E701300A28AC
:106A4000E8D14FF0FF30EDE7402C002038B5084B7F
:106A50000125D3F810441D7004B938BDE3685D7199
:106A6000236820465B689847E3681C68F4E700BF2A
:106A7000402C002030B5C38885B004460D4633B1A4
:106A8000144A00921449154A284600F07AFB217AEC
:106A900005291DD0637A4BB1A088FFF733FE104B58
:106AA000104953F82020284600F06BFB227A0E4B49
:106AB000A08853F8222003920021FFF707FE039AD3
:106AC0000A490346284605B0BDE8304000F059BBEE
:106AD00005B030BD98C0020080C0020078C002003E
:106AE00004C102009DC0020028C10200A0C0020033
:106AF00007B503460846197A052911D05B7A2BB1F0
:106B0000094A0A49019000F03CFB019808490190AC
:106B100000F037FB019803B05DF804EB00F026BBF2
:106B2000002AF8D0F2E700BF98C002009DC0020022
:106B300049C202002DE9F04385B01F460C9D002399
:106B400095F80C902B7306460C469046294638461D
:106B5000FFF790FFB8F1060F09D8DFE808F004123C
:106B6000181F283340003146284600F00AFB002257
:106B700029463846FFF7BCFF85F80C9005B0BDE804
:106B8000F08322683146284600F0FBFAEFE7D4E9AB
:106B900000233146284600F0F4FAE8E7A3680093A2
:106BA0003146D4E90023284600F0EBFADFE7E3683A
:106BB0000193A36800933146D4E90023284600F0EE
:106BC000E0FAD4E723690293E3680193A368009392
:106BD0003146D4E90023284600F0D3FAC7E76369B9
:106BE000039323690293E3680193A36800933146FA
:106BF000D4E90023284600F0C4FAB8E708292DE9B3
:106C0000F74F80460E4617461C463DD800251B7B95
:106C10002573214610460193FFF72CFFDFF88CA067
:106C2000DFF88CB0AE4232D918F80520594620461C
:106C300000F0A7FA0135082DF4D11B49DFF874A044
:106C4000DFF874B0204600F09CFA4FF000094E4582
:106C500024D918F809507E2D1ED8284604F0A2FD2C
:106C6000002814BF2A462E225946204600F089FAF1
:106C700009F10109B9F1080FE9D10122214638468D
:106C8000FFF736FF019B237303B0BDE8F08F514639
:106C9000204600F076FACDE72E22E5E75146204661
:106CA00000F06FFAE4E700BFB4C00200B0C0020019
:106CB000AAC00200B2C00200B6C0020070470000C5
:106CC00007B5044B0093044A4023FFF7BCFB03B015
:106CD0005DF804FB1D6D0200F930002030B50C4D4D
:106CE0000FCD89B06C460FC495E80F0084E80F0003
:106CF0000623084800930022694601F0FDFD08B113
:106D000000F048F8044B00221A7009B030BD00BFF3
:106D10003CC10200E82A0020F830002038B50D48B8
:106D20000D4C0E4D002323700378EB5CD2B263B19F
:106D3000043002F0D1FB08B100F02CF8084B1A78AF
:106D400012B12378002BFBD038BD0C3002F072F961
:106D5000F1E700BFE82A002039310020F831002097
:106D6000F830002008B50848084A0378D35C33B1EE
:106D7000043002F015FBBDE80840FFF7AFBF0C3050
:106D800002F0E2F8F7E700BFE82A0020F83100201F
:106D9000FFF7A4BF1FB50021039001AA44F2010030
:106DA000CDE9011100F004F805B05DF804FB000026
:106DB00038B572B6FFF74AFEFFF7C4FC0028FBD1D6
:106DC000104B114C114D1249E41AE408240444F00C
:106DD0000100FFF701FED5F8F030DB0700D500BE5B
:106DE0000C4944F00200FFF7F7FDBFF34F8FEA684C
:106DF000094B02F4E0621343EB60BFF34F8F00BF17
:106E0000FDE700BF74BF0200A4BF020000ED00E078
:106E100073C102007FC102000400FA0508B50A48E8
:106E200000F08CF8094AD2E90031C018084BD3E9C8
:106E3000002341F10001904271EB030303D210F1F2
:106E4000807041F1000108BDFC2A00204031002083
:106E50005831002037B505460C460A4801A900F014
:106E60008DF860B10570446001A9064800F0B0F8E3
:106E700018B1054800F066F8002003B030BD0420CA
:106E8000FBE700BF48310020FC2A002038B5037F13
:106E900004460D4683B98261FFF7C0FF23692818B5
:106EA00041F10001C4E9020103B12561214600203E
:106EB000BDE83840FFF7CEBF002038BD00230146B3
:106EC00003770120FFF7C6BF70B5EFF3108672B6E7
:106ED0000C4A946801239CB993600B4B0B4DD3F87B
:106EE000801029401160C3F88050D3F8841051609D
:106EF0004FF0FF32C3F88420047006B962B670BD4B
:106F00000370FAE76031002000E100E0FC06FFBDFD
:106F1000084B9A6810B55AB150B9EFF3108172B6A8
:106F2000054A1C6814605C685460986001B962B6D8
:106F300010BD00BF6031002000E100E00368D3F81D
:106F40000405704790F90430002B09DB5A09012130
:106F500003F01F0301FA03F34032024941F82230E3
:106F6000704700BF00E100E0024B034A1B68106855
:106F7000184700BF743100206C31002037B550E84D
:106F8000013F9DB2C48925448489A54228BF2D1B99
:106F90000489A54202BFBFF32F8F002207E0C5EA94
:106FA000030540E80154002CE9D14FF001028DF8AF
:106FB00003200193019A0A609DF8031001F0FF037A
:106FC00021B1006810FA82F003B030BD1846FBE72B
:106FD0000A884B889A4209D150E8012FC2EA02423E
:106FE00040E80123002BF7D10120704700207047B3
:106FF00001F01F024B090121914000EB830000F0DA
:107000001EB801F01F0301229A404B0900EB8300D8
:10701000D14300F02CB84B0901F01F0150F82300B8
:10702000C84000F00100704710B5034653E8000F58
:107030000A4643E8002494F0000FF7D110BD10B5C4
:10704000034653E8002F42EA010043E8000494F0AD
:10705000000FF6D110BD10B5034653E8000F00EA4B
:10706000010243E8002494F0000FF6D110BD10B5E2
:10707000034653E8002F02EA010043E8000494F0BD
:10708000000FF6D110BD10B5034653E8002F02EBF8
:10709000010043E8000494F0000FF6D110BD10B5D4
:1070A000034653E8002FA2EB010043E8000494F0EC
:1070B000000FF6D110BD0121FFF7C1BF0021FFF77E
:1070C000CABF10B590B1D0E9012301689B1ADBB2A9
:1070D0000A60013BDBB2FF2B026802D10020107175
:1070E00010BD11684C1C14600B70F2E70E20F7E71E
:1070F00037B5054600240DF107008DF80740FFF76E
:10710000E3FE2A686B68116899420ED9481E106028
:1071100011F8013CEC68298A01FB0344AB68117942
:107120001B1ADBB2994238BF13719DF80700FFF7B5
:10713000EFFE204603B030BD37B5054600230DF104
:1071400007000C468DF80730FFF7BEFE2A6813686B
:10715000591C1160E968641A298AB4FBF1F41C70A7
:107160009DF80700FFF7D4FE03B030BD826810B56C
:1071700004462AB143690168006998470023A36067
:1071800010BD0EB403B5039921B104AB01AA01935C
:1071900000F076F802B05DF804EB03B070470A29FE
:1071A00038B504460D4602D10D21FFF7F8FFA3685C
:1071B0002268591CA160D554D4E901329A4204D303
:1071C0002046BDE83840FFF7D1BF38BD2DE9F84F64
:1071D0009846DDE90A43154682460F460A464FF0B7
:1071E0000109AA420FD2C14538BFC14613F0010BB5
:1071F00001D16CB900240126B8F1010F1BD908F1A7
:10720000FF386E43F8E709F10109B2FBF5F2E8E750
:107210009B070ED5B8F1000F0CBF30262026A145E4
:10722000E9D2013C31465046FFF7B9FF002CF6D1B8
:10723000E0E72026F3E7B7FBF6F39D42E1D9DFF85C
:107240003C80B7FBF6F3504618F8031006FB1377A3
:10725000FFF7A5FF3346AB42B6FBF5F6F1D2BBF123
:10726000000F02D00CB1A14501D3BDE8F88F202159
:107270005046013CFFF793FFF4E700BF96C10200C0
:107280002DE9F74F054617468846002900F03E8154
:1072900018F8011B49B92B7B002B00F037812846D9
:1072A00003B0BDE8F04FFFF761BF252940F0B7807C
:1072B000002698F800302D2B424608F1010823D013
:1072C000302B24D02B2B25D000242A2B02F10101B6
:1072D00023D13B681A1D1B683A601C440A46137888
:1072E0002E2B26D101324FF0000A104610F8011B58
:1072F000A1F1300CBCF1090F1DD80A2303FB0A13BE
:10730000A3F1300A0246F0E746F00106D1E746F065
:107310000206CEE746F00406CBE711F8013CA3F1E4
:1073200030000928DBD80A2202FB0434303C0A462C
:10733000CBE74FF0000A12F8011B01F0FB006828B0
:107340009046F8D0782909D86F290CD8632962D0E3
:1073500022D8252963D0582900F0888098F8003079
:10736000002B95D197E770390829F7D801A353F876
:1073700021F000BFE77402005D7302005D7302003C
:107380007D7402005D7302005B7402005D73020095
:107390005D7302006D740200642901D06929DDD19A
:1073A0003A68D2F80090111D89EAE9723960A2EBBF
:1073B000E9724FF0010B092A35DCD34538BFD346BB
:1073C0002CB1B9F1000F01DB720700D5013CB30706
:1073D00002D5BAF1000F03D0F00701D44CBB002452
:1073E000B9F1000F2DDAC9F100092D212846FFF768
:1073F000D6FE06F00302022A04D1BAF1000F01D131
:107400001CBB0024CDE9004653460A2249462846C3
:10741000FFF7DCFEA2E73B681A1D19783A602846A0
:10742000FFF7BDFE9AE70A230BF1010BB2FBF3F263
:10743000C1E7A345D4D220212846013CFFF7AFFE87
:10744000CCE77107D5D52B21D0E7A345DAD230217F
:107450002846013CFFF7A3FED2E73968CDE9004694
:107460000A1D3A6053460A220968D0E739680A1DA6
:107470003A60CDE9004653461022F5E73B681A1DF5
:107480003A6016F00106D3F8009024D1B9F1000F4C
:1074900003D0484604F0FCF90646B4421DD809F171
:1074A000FF3919F8011F00293FF458AF2846FFF7AC
:1074B00076FEF6E728460136FFF771FE19F806104A
:1074C0000029F7D1A642BFF449AF20212846013C4C
:1074D000FFF765FEF6E70026F0E720212846013C8D
:1074E000FFF75DFED9E73B681A1D3A603021284658
:1074F0001C68FFF754FE78212846FFF750FE002253
:107500000823CDE900322146102280E703B0BDE810
:10751000F08F00BF2DE9F84FB0F806A04579D2F8FA
:1075200000B09DF828900AFB05F5043D88460BEB5A
:107530000301A94203F1040488BFA5EB030BB4FBCC
:10754000FAF607460AFB1644C2F800B04EB9AAEB99
:1075500004055D4528BF5D46BBF1000F04D1BDE8C1
:10756000F88F3F68013EF1E7043408EB06003C4425
:107570002A46B9F1000F0DD02146ABEB050B04F004
:107580003CF9DA452E443F6855464FF0000428BFC9
:107590005D46E1E701462046EFE7FFF792BDF8B50B
:1075A00046790146721E0546002393422D6803D397
:1075B0000024A64202D8F8BD0133F6E70F6828463A
:1075C000FFF7BAFD01343946F3E72DE9F843068A9F
:1075D000CD1C0746FFF78CFD043E35440446B5FB41
:1075E000F6F5F0B14FF48073EDB28380C680013DB3
:1075F000076081464FF00008A84512D23846FFF7D1
:1076000077FD064648B163790133637108F10108DB
:10761000C9F8000007608146EEE72046FFF7BFFF8C
:1076200034462046BDE8F88301210430FFF72BBD26
:1076300010B5012104460430FFF731FDC0B220B976
:107640002046BDE81040FFF7AABF10BD1FB503924A
:107650000022009203AAFFF75DFF05B05DF804FB6E
:107660001FB503920122009203AAFFF753FF05B052
:107670005DF804FB836800225A60C3E904229A6023
:10768000DA601A6070470B684A684360934208BF2B
:107690000023016008BF43607047436843B102683C
:1076A000916852680B449342436004BF00234360D7
:1076B0007047000030B50D4C94F858500124AC4090
:1076C0004FF0A04585B0C5F80C45CDE90001CDE9E6
:1076D000022307480022694602F0ECF820B105B009
:1076E000BDE83040FFF756BB05B030BD7831002013
:1076F000BCC10200F8B52C4B93F82340002C50D1AC
:1077000046B2002E41DB012583F823501D1900F0FD
:107710007F0785F82870651C53FA85F50F0E85F8EC
:107720002870A51C53FA85F50F0C85F82870E51C08
:1077300053FA85F50F0A85F82870251D53FA85F54B
:10774000402885F828102AD048280CBF8721FF211F
:10775000023A012A94BF0522012283F82420002E38
:1077600004F1050453FA84F4A8BF93F824300F4AB7
:1077700084F82810B8BF01230E33A2F11000DBB249
:107780000621FFF797FF0020F8BD022483F823406D
:1077900077249C624FF47F449C850624B6E79521AC
:1077A000D6E71120F0E700BF78310020B03100208B
:1077B0002DE9F843524CE68B40F2D915AE4238D051
:1077C000B6F5ED7F08D2A6B140F2C715AE4229D07A
:1077D0000023E383032055E0B6F5F07F4FF000016E
:1077E00009D0B6F5F67FF3D184F823101970E18340
:1077F00042E0A58AE582E68AFF255EB9414A84F81F
:10780000285002230121A2F11000FFF753FF4FF48B
:10781000F67368E0002684F8285003252684268322
:1078200084F8235044F62065042794F82360032E3F
:107830000FD0238B934243D3E38A324A013BE38246
:1078400001210223A2F11000FFF734FF4FF4F0737F
:1078500049E0268C0136B6B2AE4226840ED8844664
:10786000002943D010F8016BFF2E0DD0FE2E0ED054
:1078700005221A700023E383022003E0022018701F
:107880000023E383BDE8F8830139C9B2E7E74E1E60
:10789000F1B291420E4684F8237028BF16464FF08D
:1078A00000084645D4F80CE003D826837644E66009
:1078B000BBE71CF8019F0EF8089008F10108F0E7FB
:1078C000D51AADB2F02D28BFF025EBB2E2680E4814
:1078D0000121FFF7EFFEE3682B44E360238B1D4497
:1078E000258340F2D913E3830120CBE7054A102317
:1078F0000121A2F11000FFF7DDFE40F2C713F2E70D
:1079000078310020B0310020A031002010B5164B96
:1079100093F822400CB393F82240032C1FD102B3FA
:10792000042483F822409C7A9A82240758BF490293
:10793000012AC3E90301DA824FF000044FF001028B
:1079400014BF522051209C83FFF7D4FE034610B190
:10795000FFF720FA2346184610BD0823FBE7112342
:10796000F9E70723F7E700BF7831002038B5184B57
:10797000154693F822202AB393F82220032A23D114
:1079800025B3052283F822209A7A9D82140758BFD6
:1079900049020024012DC3E90301DD829C8308D143
:1079A0002A465820FFF7A6FE08B1FFF7F3F900209A
:1079B00038BD02F00702012A0FBF592001222946D3
:1079C000D720EFE70820F3E71120F1E70720EFE7E2
:1079D00078310020F0B5324C94F8222089B00D4661
:1079E00002F0FF03002A57D1002957D0C278FF2A9E
:1079F00054D04178FF2951D00778FF2F4ED080789E
:107A0000FF284BD002F5E0764FF0A04C4FF0030E6C
:107A100084F858204CF826E0012606FA02F2CCF849
:107A20000825FF228DF803204FF60672ADF80420DA
:107A30004FF080628DF800008DF802100292194814
:107A4000194A8DF801706946ADF80C3001F0B0FDAF
:107A500008B1FFF79FF9A37A256023F00F03A37203
:107A6000FF2384F82830114B114884F82260CDE9B7
:107A700004360025103306932A460A2304A90793E7
:107A800084F8235001F016FF034610B1FFF782F986
:107A90002B46184609B0F0BD0823FAE70723F8E79C
:107AA00078310020B8C10200F97A0200A03100202C
:107AB000BCC1020010B50E4C94F82230A3B194F86A
:107AC0002230032B12D10B4801F0A6FE94F8583057
:107AD0004FF0A04203F5E073002042F8230084F841
:107AE000230084F8220010BD0820FCE71120FAE7EB
:107AF00078310020BCC10200F7B5AD4C0146E68AE2
:107B0000C0680D7C3EB994F85820012393404FF093
:107B1000A042C2F8083594F823707B1E012B6FD861
:107B2000496891F800C0AA1FBCF14C0FD2B200F115
:107B3000060303D14AB1EA1FD2B2C31D1946154646
:107B40000B4645B9BCF14C0F20D1013B012507E0A4
:107B5000013DEDB2F4E71A78FF2A01F10101F7D0F7
:107B6000022F49D1012284F823201A7812F0FE0F47
:107B700042D194F824308F4A0E33DBB20621A2F1B1
:107B80000A0003B0BDE8F040FFF794BD94F822303E
:107B9000012B2FD094F82210012204298DF8052002
:107BA000CBB216D004D8013B934207D903200DE095
:107BB000052BFBD102238DF804300CE003238DF854
:107BC000045084F82230FFF775FF20B1FFF7E2F888
:107BD00001E08DF8042094F85820012393404FF0E1
:107BE000A042C2F80835032384F82230236801A894
:107BF000984794E02B46B3E7002284F823201846E8
:107C000094F82230D9B2013B042B00F2CD82DFE898
:107C100013F005000A00CB027801C201022384F8A8
:107C200022300023A383A18B0378B1F50E7F00F0EF
:107C3000D0802CD840F21322914272D0B1F5057F4A
:107C400008D2002961D0B1F5047F53D00023A3836B
:107C500006216CE040F21922914200F08A8040F245
:107C600026229142F2D1580740F1E480A37A012202
:107C700062F30203A372238C01339BB2B3F5FA6F54
:107C8000238440F29B800023A38302214FE040F233
:107C90006122914200F0DF8015D840F24D229142DE
:107CA00000F0C88040F253229142CFD113F0FC0F74
:107CB0003AD1D0F801301BBA5A0042BFA37A43F040
:107CC0000803A3728BE040F26B22914200F0D58052
:107CD000B1F51C7FBAD101AB10222946FFF768FD30
:107CE00001281CD99DF80410002900F0D180002340
:107CF000A3831CE0012200214020FFF7FBFC08B118
:107D0000FFF748F840F2132308E001224020FFF774
:107D1000F1FC08B1FFF73EF84FF40473A38303B0FE
:107D2000F0BD13F0FC0F18D00023A383042100231F
:107D300094F858208DF80430032384F8223001236E
:107D400093404FF0A0428DF80510C2F808351A4B49
:107D50004FF08042C3F8242548E703224FF4D57141
:107D60004820FFF7C7FC08B1FFF714F840F21923C9
:107D7000D4E75D0707D4A27A032161F3020213F06E
:107D8000FC0FA272D0D100232384A37A03F007034F
:107D9000032B0CBF4FF0804100210222E920FFF7A6
:107DA000A9FC08B1FEF7F6FF40F22623B6E700BFB4
:107DB00078310020B0310020003000400222002144
:107DC0004120FFF797FC08B1FEF7E4FF4FF40E7374
:107DD000A4E713F0FC0FA7D1D9073FF54CAFA37A66
:107DE00003F00703032B3AD001224FF40071502017
:107DF000FFF780FC08B1FEF7CDFF40F261238DE76D
:107E0000238C01339BB2B3F5FA6F23843FF63BAF6B
:107E1000A37A03F00703032B0CBF4FF0804100212E
:107E20000222E920FFF766FC08B1FEF7B3FF40F23B
:107E30004D2373E713F0FC0F7FF476AF13F00101CD
:107E4000DED102227A20FFF755FC08B1FEF7A2FF2F
:107E500040F2532362E713F0FC0F7FF465AFB04BA1
:107E6000E360012200214920A282FFF743FC08B110
:107E7000FEF790FF40F26B2350E713F0FC0F7FF406
:107E800053AF013D4FF41C730130EDB2E36122E7C3
:107E900094F848309B09012B24D0DB072FD494F8A9
:107EA0004F3094F8502094F852009B0003EB92134B
:107EB00094F84E20920202F440620133134494F885
:107EC0005120520002F0060202EBD01294F84D004D
:107ED00000F00F0007380244934063604FF40073D2
:107EE000238104E794F8513094F85020013303EBD8
:107EF000022394F84F2003EB02439B02EDE70B466D
:107F0000EBE7A38BB3F5267F0FD040F2A22293427A
:107F10003AD0002B3BD1037813F0FC0F13D1013D75
:107F20004FF426730130EDB2E36101AB4FF4007200
:107F30002946FFF73DFC01287FF6F1AE9DF80410BD
:107F4000A9B10023A383032284F822200022012365
:107F5000626184F8232094F858208DF804308DF85D
:107F6000051093404FF0A042C2F808353EE6A38AC0
:107F7000012B09D901224C20FFF7BCFB08B1FEF709
:107F800009FF40F2A223C9E60021A183DBE7002319
:107F9000A3830621D7E7A28BB2F53B7F00F0A38035
:107FA00027D840F2C3239A423ED0B2F5317F05D2A2
:107FB000002A41D00023A3830621A1E040F2D3236D
:107FC0009A4202D0B2F5397FF4D1268BE068B6F53B
:107FD000007F76D3534A00F500700323E06001214F
:107FE000A2F1100084F82330FFF764FB4FF43B73D9
:107FF00094E6B2F5487F4FF0000300F0B380B2F58D
:108000004C7F00F0C88040F20A318A42D2D1AB42A4
:1080100080F08B80C25C002A00F0A280002384F8EC
:108020002330013EE68220E0037813F0FC0F1AD0E3
:108030000023A383042163E0037813F0FC0FF9D13C
:10804000A37A03F00703012B0DD0A38A012B0AD9D1
:10805000216901225920FFF74DFB08B1FEF79AFE76
:1080600040F2C3235AE6A38AE382E28AA38A7AB95A
:10807000012B40F296802B4A4FF6FF5323850221B5
:108080000323A2F11000FFF715FB4FF4487345E6F8
:10809000002222830422012B84F823204FF0FF02C8
:1080A0008CBFFC23FE2384F828201E4A84F8293044
:1080B00002231946A2F11000FFF7FCFA40F2D32385
:1080C0002CE6C6F50075ADB2F02D28BFF0250123D2
:1080D000E9B2144A3044FFF7EDFA238B1D4425839F
:1080E0004FF439731AE694F83A3003F01F03052B66
:1080F0004FF0000218D00B2B01D00D2B98D1A2838A
:1081000002238DF80430032384F82230002384F8FE
:108110002330636194F858208DF80510012320E77F
:10812000C0310020B0310020228494F82330032B8A
:108130007FF477AF238C01339BB244F620629342E5
:10814000238403D90023A3830221D9E7194A1023EA
:108150000121A2F11000FFF7ADFA40F20A33DDE58C
:10816000013354E72384032384F82330238C013321
:108170009BB244F6206293422384E3D80D4A102335
:108180000121A2F11000FFF795FA4FF44C73C5E5F9
:10819000C25C32B90133AB42FAD394F82330032BDB
:1081A000E4D00021A183ABE7032003B0BDE8F04099
:1081B000FEF7F0BDB0310020064B93F82220032AD1
:1081C00005D093F82200003818BF01207047002026
:1081D000704700BF78310020044890F82230022B0D
:1081E00000F1040098BF0020704700BF78310020E4
:1081F00019B1012905D00620704702B11170002085
:10820000704712B104301060F9E7072070478069A9
:10821000704708B5FFF7D0FF0028FBD108BD00006C
:10822000F0B51B4B1B68834285B005460C4603D056
:108230001124204605B0F0BD8669FFF7BDFF002878
:10824000F6D194E8070006F10C0787E80700A2883A
:108250002168A068FFF78AFB044640B9B36833B9C8
:10826000FFF7D7FF0B4B1B78002B18BF0D24B3680B
:10827000002BDED0002CDCD04FF48172ADF804204E
:10828000B2690297039201A928469847D1E700BF37
:10829000D4310020D8310020F0B51B4B1B6883423D
:1082A00085B005460C4603D01124204605B0F0BD2C
:1082B0008669FFF781FF0028F6D194E8070006F1F0
:1082C0000C0787E80700A2882168A068FFF71EFB5B
:1082D000044640B9B36833B9FFF79BFF0B4B1B78DB
:1082E000002B18BF0D24B368002BDED0002CDCD08F
:1082F0004FF48172ADF80420B2690297039201A98C
:1083000028469847D1E700BFD4310020D83100205B
:10831000F0B5134F3B68834285B0054603D0112466
:10832000204605B0F0BD8669FFF746FF0028F6D16C
:10833000FFF7C0FB044600B93860B368002BEFD0EC
:1083400001228DF80420221E18BF01228DF805207D
:1083500000220292B269039201A928469847DFE7FA
:10836000D43100202DE9FF410369B3F5007F0546B4
:108370000E4629D1DFF86080D8F8003033BB87691A
:10838000C8F80000B960BA6111491430FFF722FB48
:10839000044630B9A6B9FFF73CFF0E4B1B787BB102
:1083A0000D240023C8F8003056B14FF480720293B8
:1083B000BB690393ADF80420BB6801A92846984720
:1083C000204604B0BDE8F0810624F9E71124F7E760
:1083D000DD830200D8310020D4310020F0B5294AD5
:1083E0004378294F137002783D68012AAC6985B043
:1083F000064627D0022A39D0002A3CD12BB1284684
:10840000FFF786FF08B1FEF7C5FCFFF7E5FE03683E
:1084100023604FF4007363603B689B699B687BB18A
:10842000737800229B1A18BF01238DF804208DF861
:108430000530A36903930292A36801A928469847CF
:1084400005B0F0BDA268002AFAD00221003B18BF97
:1084500001238DF804108DF8053004F10C0302930C
:10846000A369039301A928469047E9E7A268002A77
:10847000E6D00321EAE7032005B0BDE8F040FEF7AF
:1084800089BC00BFD8310020D43100204FF0805388
:10849000D3F83001421C04BF4FF0704393F8E00F53
:1084A000831F5842584170474FF0704393F8E02FB4
:1084B000062A09D1D3F8E83FC3F30313033B032B88
:1084C00002D8024AD05C704700207047E8C1020021
:1084D00008B5FFF7DBFF40B14FF080538F4AD3F868
:1084E0002433C3F30423C2F84035FFF7DDFF10B196
:1084F0008B4B8C4A5A67FFF7C9FF48B14FF0805346
:108500004FF08042D3F84432C3F34233C2F83C35D3
:10851000FFF7CAFF30B1844AD2F8FC3023F08073F1
:10852000C2F8FC30FFF7B2FF40B14FF080430022A9
:10853000C3F80C21C3F81021C3F83825FFF7B4FFA6
:1085400020B14FF080430322C3F8A025FFF7ACFF12
:1085500060B1764B0522C3F810260122C3F88826A5
:108560000022C3F818263F22C3F814264FF0805388
:10857000D3F83021511C09BF4FF07043D3F8343188
:1085800093F8E02FD3F8E83F08BFC3F30313062A9C
:108590004DD1033B032B03D8654AD35C002B46D057
:1085A0004FF08052634BD2F80414C3F82015D2F870
:1085B0000814C3F82415D2F80C14C3F82815D2F8FF
:1085C0001014C3F82C15D2F81414C3F83015D2F8CF
:1085D0001814C3F83415D2F81C14C3F84015D2F897
:1085E0002014C3F84415D2F82414C3F84815D2F85F
:1085F0002814C3F84C15D2F82C14C3F85015D2F82F
:108600003014C3F85415D2F83414C3F86015D2F8F6
:108610003814C3F86415D2F83C14C3F86815D2F8BE
:108620004014C3F86C15D2F84424C3F87025FFF742
:108630002DFF48B14FF080534FF08042D3F85832AD
:1086400003F04F03C2F8E43EFFF720FF48B14FF0BC
:108650008043D3F80024D20744BF6FF00102C3F86F
:1086600000244FF08053D3F83021062A0ED1D3F8DE
:108670003431033B032B02D82F4AD35C33B12F4A4A
:10868000D2F83C3743F48063C2F83C37264AD2F82C
:10869000883043F47003C2F88830BFF34F8FBFF3C4
:1086A0006F8F4FF01023D3F80022002A03DBD3F89A
:1086B0000432002B2EDA224B0122C3F80425D3F812
:1086C0000024002AFBD04FF010221521C2F800121E
:1086D000D3F80024002AFBD04FF010231522C3F852
:1086E0000422174BD3F80024002AFBD00022C3F841
:1086F0000425D3F80024002AFBD0BFF34F8F0A498A
:10870000104BCA6802F4E0621343CB60BFF34F8F93
:1087100000BFFDE70C4B0D4A1A6008BD0030014058
:1087200000C007400DF0ADBA00ED00E00050004081
:10873000E0C1020000C00040E4C10200001000409F
:1087400000E001400400FA05042B00200090D00353
:1087500038B5074C051E04F1080318BF1C462368F2
:108760002BB11A6822605B6828469847F7E738BD46
:10877000E431002020B9054B01225A70FFF7E8BF11
:10878000012802D1014A9070F8E77047DC310020DF
:1087900020B9034B01225A70FFF7DABF704700BFC0
:1087A000DC31002038B50E4C2378B3B90D48636036
:1087B000A3602361E36000F0E7F8054601F084FD63
:1087C00008B900F0EDF801232370074BD3F800340B
:1087D0000BB10123A370284638BD8525F5E700BFFE
:1087E000DC310020758702000000014037B50D4CD8
:1087F00000230DF107008DF80730FEF765FBE368F5
:10880000013BE360E36833B9074BD3F8005415B973
:1088100000F0D8F8A5709DF80700FEF779FB03B0CB
:1088200030BD00BFDC31002000000140012813B53D
:108830000CD0032820D038B9134B0122C3F8802074
:10884000BFF34F8FBFF36F8F02B010BD0F4C0023EB
:108850000DF107008DF80730FEF736FB23780BB9D2
:10886000FFF7A0FFE3689DF807000133E3600123F1
:10887000A370FEF74DFBE7E700F092F802B0BDE809
:108880001040FFF7B3BF00BF00E100E0DC31002083
:108890001FB503788DF800304368019383688DF825
:1088A0000830C368054A0393054B684653F82130E6
:1088B00052F82110984705B05DF804FBF031002014
:1088C000F43100201FB503788DF800304368019320
:1088D00083688DF80830C368054A0393054B6846E2
:1088E00053F8213052F82110984705B05DF804FB89
:1088F000F0310020F4310020F0B5194B90F800C0A1
:1089000091F81DE043F82C20164B16460A6943F8EF
:108910002C20154B03F80CE00C4607460FCC89B011
:108920006D460FC594E80F0085E80F00CDF810C024
:10893000BEF1000F09D0002E0C4A694608BF32462E
:10894000381D00F06BFC09B0F0BD002E084A6946E6
:1089500008BF324607F10C0000F042FAF3E700BF0F
:10896000F4310020F0310020F8310020918802001D
:10897000C588020000F18040002382B003600368D4
:108980000193019B02B07047044A137923B9012176
:10899000106091801846704785207047FC31002098
:1089A000074B1A68D20704D4C02283F8002301229F
:1089B0001A604FF080430122C3F81825704700BFAA
:1089C00000E100E04FF0804208B50223C2F808330E
:1089D0004FF48270FFF7CEFF0123D360D2F8183432
:1089E000DB03FBD408BD00004FF0804110B5D1F887
:1089F000003163B14FF48070FFF7BCFF0D4B587925
:108A00000122C1F8082310B95A711B6898474FF02A
:108A10008042D2F8043163B14FF48270FFF7AAFFAD
:108A20000223C2F80833034BBDE810401B68012045
:108A3000184710BDFC31002000F1804000F5C04017
:108A4000002382B0036003680193019B02B070476A
:108A5000800000F1A040D0F8002722F44032C0F896
:108A60000027D0F8003743EA0141C0F800177047EB
:108A70002DE9F74F00244E4D01944FF480720121EF
:108A800002F1804303F5C04390B21B68012B06D16D
:108A9000D5F804330B4202D0FFF7CEFF0C4304326B
:108AA000B2F5907F4FEA4101EAD1414BD3F87C31D6
:108AB000012B0CD14FF4BE70FFF7BEFF4FF0A04367
:108AC00044F00044D3F820250192C3F82025E3B2F6
:108AD000D3B1384F00250126344210D0AB0003F14A
:108AE000804303F5C043D3F81005D3F8101557F8A9
:108AF000253023B1C1F30141C0F30420984701356B
:108B0000082D4FEA4606E7D1002C48DA294D4FF0F0
:108B1000A048294E4FF00009012716F9013B5A1CC5
:108B200031D0C3F3C20202A90A44DCB212F8042C09
:108B300003F03F0A03F0070307FA03F31A4222D0B7
:108B40000AF5E073504658F82330C3F3014BBBF1EC
:108B5000020F0CBF03210221FFF77AFF07FA0AF385
:108B6000C8F8203505EB0A0393F9303055F8233067
:108B70004BB1A109032904D0BBF1020F12D1012985
:108B800001D15046984709F10109B9F1040FC4D148
:108B9000D8F820350193C8F82035002BB9D103B09F
:108BA000BDE8F08FBBF1030FEDD10229E8E700BF6C
:108BB000006000400432002054320020014B1B684A
:108BC000184700BF603200200E4B984237B50C4664
:108BD00002D0002003B030BD00230DF107008DF856
:108BE0000730FEF771F9084B1D7915B901221C6099
:108BF0001A719DF80700FEF78BF9002DE9D01120BE
:108C0000E8E700BF0020004060320020034B98429C
:108C100001BF034B00221A601A7170470020004008
:108C2000603200200023435082B043580193019BDF
:108C300002B070470A4610B54FF48E71FFF7F2FF8D
:108C4000136A9168C95C136A01331362C0F81C157A
:108C500010BD8B690A4610B54FF4847123B9FFF734
:108C6000E1FFD0F8183510BDFFF7DCFF536AD1687B
:108C7000D0F81805C854536A01335362F3E7000073
:108C80001FB501238DF80030044BCDE90110D3E965
:108C900000126846904705B05DF804FB683200207A
:108CA00030B54D4DD5F804339A0585B051D5D5F87A
:108CB0002431002B4DD04FF492712846FFF7B2FFBC
:108CC0004FF40173C5F80833444B93F829200AB9CF
:108CD00001226A60404902228DF80020D1F88024E8
:108CE000C1F8802403929A690292DA680192002204
:108CF000C3E906226846D3E9001290473648D0F807
:108D00001C315BB1354A5169136A99424DD992F8C9
:108D10002830002B49D11146FFF78CFF2E48D0F8A0
:108D20004431002B56D04FF4A271FFF77BFF2B4B41
:108D300093F829200AB1012202609A69002A49D0D9
:108D4000586AD96800229A6105B0BDE83040FFF743
:108D500097BFD5F804335B07D0D5D5F80831002B81
:108D6000CCD01E4C1C482146FFF773FF636AA269F2
:108D70009A42C3D1E369E1684BB1A3612369E3601F
:108D80000023606AE3616362FFF77AFFB6E794F855
:108D900029300BB901236B600F4B4FF40172C3F8FC
:108DA00008230023606AA361EEE70B484FF48E713D
:108DB000FFF738FF5369002BB0D0516902910023AF
:108DC00091688DF80030019153616846D2E9001333
:108DD0009847A3E705B030BD00200040683200206E
:108DE0002DE9F843534D90F804802C2303FB0853DE
:108DF000064693F82A300C469146002B40F09680A8
:108E00004D490068FFF7E0FE0746002840F09080DB
:108E100022683068511C0BD04FF0A04101239340D1
:108E2000C1F8083502F5E0734FF0030C41F823C098
:108E300061684B1C1FBF01F5E0734FF0A04C4FF071
:108E4000000E4CF823E0A369C0F8243594F814C050
:108E5000637DBCF1010F4CEA0303C0F86C35C0F828
:108E60001415C0F80C251DD1A268531C1FBF02F5B4
:108E7000E0734FF0A0414FF0000C41F823C0E368CD
:108E8000591C0BD04FF0A04C01219940CCF808158B
:108E900003F5E0714FF0030E4CF821E0C0F80835FF
:108EA000C0F810252C2202FB08F2AB18C3F804907E
:108EB0002369AB50B9F1000F20D04FF48E71247F9D
:108EC000FFF7B0FE4FF4A2713068FFF7ABFE3268D7
:108ED0001A4BC2F80433130B42F307326101002A24
:108EE000C9B21EDB1648841884F800130121520908
:108EF00003F01F0301FA03F340F822303368042221
:108F0000C3F800252C2303FB08530022C3E90622E3
:108F100083F829205A61012283F82A203846BDE8C7
:108F2000F883084A03F00F03D154E7E70827F5E771
:108F30001127F3E768320020A18C020080000200B4
:108F400000E100E014ED00E0F8B503680579304C6D
:108F50000022C3F800252C2202FB05425268A2B170
:108F60002C4AC3F808231A0B43F30733002B0CDBFE
:108F700002F01F015B0901228A402033264941F893
:108F80002320BFF34F8FBFF36F8F0068D0F80C65BD
:108F9000D0F81415D0F80835D0F810254FF0FF3769
:108FA000BE42C0F8147518BF06F5E076C0F80C751F
:108FB000C0F80875C0F810751EBF4FF0A0474FF0FD
:108FC000020C47F826C04E1C1FBF4FF0A04601F50B
:108FD000E071022746F82170511C1FBF4FF0A041DD
:108FE00002F5E072022641F822605A1C1FBF03F509
:108FF000E0734FF0A042022142F82310FFF706FE73
:109000002C2303FB0544002384F82A306360F8BD59
:10901000683200208402020000E100E00279044B83
:109020002C2101FB02335869003818BF012070471A
:10903000683200202DE9F84F064690F804808946F2
:109040009246FFF7EBFF044600283CD1204F2C2529
:1090500008FB057B4FF48E71CBF814A0CBF8089079
:10906000CBF820008BF828003068FFF7DBFD306874
:10907000012383605946FFF7DDFDDBF804305D46D0
:109080001BBB3068DBF814402B6A9C4211D8336854
:10909000D3F81C21002AFBD00122DA6000202C2307
:1090A00003FB087700237B61BDE8F88F95F8283033
:1090B0003BB9D0F81C31002BF8D05946FFF7BAFD68
:1090C000E2E70F20EBE71120EEE72046ECE700BFD8
:1090D000683200200023435082B043580193019B23
:1090E00002B070471FB501238DF80030044BCDE965
:1090F0000110D3E900126846904705B05DF804FB03
:10910000943200207FB5434AD2F82461002E60D00B
:1091100010464FF49271FFF7DDFF02238DF8003007
:10912000D2F88034C2F880340393D2F83C350293ED
:10913000394BDA6801920022C3E906226846D3E976
:10914000001290473348D0F8443173B14FF4A27104
:10915000FFF7C0FF304B9A693AB10022C3E90622FB
:10916000D968D0F83C05FFF7BDFF2A48D0F8203178
:10917000ABB14FF49071FFF7ADFF0123C360264BF5
:109180005A6962B1D0F84C150291002299688DF8A5
:10919000002001915A616846D3E9001290471D48AA
:1091A000D0F858319BB14FF4AC71FFF793FF1A4BD5
:1091B0005A6962B1D0F84C150291002299688DF875
:1091C000002001915A616846D3E90012904704B02B
:1091D00070BDD2F81031002BB4D04FF48871104616
:1091E000FFF778FF0C4BD2F83C0599698842A9D16A
:1091F000DC69D96864B1D2F8005225F02005C2F8C4
:1092000000521A699C61DA60DE61FFF76BFF99E733
:109210009C61FAE700200040943200202DE9F843D9
:109220005A4E90F80480242303FB0863044693F805
:1092300020300D469146002B40F0A3805449006831
:10924000FFF7C2FC0746002840F09D802A6820688E
:10925000511C0BD04FF0A04101239340C1F80835B9
:1092600002F5E0734FF0030C41F823C069684B1C12
:109270001FBF01F5E0734FF0A04C4FF0000E4CF80B
:1092800023E0AB69C0F8243595F814C06B7DBCF1C0
:10929000010F4CEA0303C0F86C35C0F80C25C0F888
:1092A00014151DD1AA68531C1FBF02F5E0734FF0BF
:1092B000A0414FF0000C41F823C0EB68591C0BD0C3
:1092C0004FF0A04C01219940CCF8081503F5E0714E
:1092D0004FF0030E4CF821E0C0F80835C0F8102517
:1092E000242202FB08F2B318C3F804902B69B35090
:1092F000B9F1000F2FD04FF488712A7FFFF7EAFEF3
:1093000020684FF49071FFF7E5FE20684FF49271EA
:10931000FFF7E0FE20684FF4A271FFF7DBFE4FF489
:10932000AC712068FFF7D6FE23681A49C3F804130E
:10933000190B43F307335201002BD2B21CDB164842
:10934000C51885F8002301225B0901F01F0102FA0C
:1093500001F140F8231023680822C3F800252423D4
:1093600003FB08660023C6E906337361012386F810
:1093700020303846BDE8F883084B01F00F015A54FD
:10938000E9E70827F5E71127F3E700BF943200204B
:10939000059102001003420000E100E014ED00E03E
:1093A000F8B5444C0579242303FB054302465B686A
:1093B0000068ABB1404BC0F8083340F30733002BD3
:1093C0004FEA10310CDB01F01F065B090121B140AF
:1093D00020333A4E46F82310BFF34F8FBFF36F8F01
:1093E000D0F8003223F02003C0F80032242303FB1E
:1093F00005439B692BB14FF4A271FFF76BFE01236C
:1094000043604FF4AC71FFF765FE0123C360242372
:1094100003FB0543D0F858110029FBD0996919B115
:10942000D0F844110029F5D00023C0F800351368A6
:10943000D3F80C75D3F81465D3F80825D3F81015B4
:109440004FF0FF3C6745C3F80CC518BF07F5E07740
:10945000C3F814C5C3F808C5C3F810C51EBF4FF044
:10946000A0434FF0020C43F827C0771C1FBF4FF0FA
:10947000A04306F5E076022743F826704E1C1FBF76
:1094800001F5E0714FF0A043022643F82160531C20
:109490001FBF4FF0A04302F5E072022143F82210F3
:1094A000FFF7B4FB242303FB0544002384F820309A
:1094B0006360F8BD943200201003420000E100E038
:1094C0000279044B242101FB02335869003818BF8C
:1094D000012070479432002001F06043B3F1005F37
:1094E0002DE9F0470646884692463BD190F8049015
:1094F000FFF7E6FF0446002836D11D4F30682425CB
:1095000005FB09754FF49071C5F814A0C5F80880E3
:10951000FFF7E0FD4FF4AC713068FFF7DBFD336817
:109520006A69A968C3F84415C3F8482501229A60FE
:109530006A68DAB9D3F82021D3F858011AB900289B
:10954000F8D00F2007E00028FBD10122DA60D3F821
:109550005821002AFBD0242303FB097700237B61D9
:10956000BDE8F0871020FBE71120F9E72046F7E778
:10957000943200207FB503788DF80430436802935D
:1095800083688DF80C30C36804930369064A8DF82C
:109590001430064B01A853F8213052F82110984797
:1095A00007B05DF804FB00BFB8320020C4320020D1
:1095B000F0B50546174615F804CB124A42F82C7050
:1095C000114A42F82C30114B0C460FCB85B06E4639
:1095D00086E80F002368009323798DF805306379BE
:1095E0008DF80630A3680293002FA389084AADF8CE
:1095F0000C3008BF3A4663463146284600F036F83C
:1096000005B0F0BDC4320020B832002010C2020004
:1096100075950200124BD3F8182182B0EAB10022EE
:10962000C3F81821D3F818310193019B0D4BD97F52
:10963000FF2907D0987F01228A404FF0A04148B10E
:10964000C1F80C2500225A771A72D3E90021064886
:1096500002B01047C1F80825F4E702B0704700BF18
:1096600000300040D0320020D83200202DE9F74FE2
:1096700090F80480644E01924FF0240909FB08F928
:1096800006EB090B9A469BF81C3007460C46002B4C
:1096900040F0B58005685D492846FFF795FA002837
:1096A00040F0AF80019B46F80930CBF804A094F855
:1096B00000E094F80CC04FF0A042012303FA0EF32F
:1096C000BCF1010F94BFC2F80C35C2F808350EF595
:1096D000E073012142F823106378FF2B1FBF9940EC
:1096E000C2F80C1503F5E0714FF0030918BF42F8FA
:1096F0002190A27808BF4FF0FF33FF2A1FBF02F569
:10970000E0714FF0A04A4FF0040B4AF821B04FF03F
:10971000240101FB086618BF914686F82020E278F4
:109720003949F27708BF4FF0FF39FF2A17D094F874
:1097300004A04FF0010B0BFA02FB4FF0A046BAF168
:10974000000F4ED0C6F80CB502F5E0724FF0030BD7
:1097500046F822B0242202FB081282F81EA0C5F8A7
:1097600008E5C5F80C35A368C5F81095C5F824358B
:10977000637B003B18BF0123BCF1020F34D0BCF166
:10978000030F34D0BCF1010F01D143F00203C5F83F
:109790005435A379C5F8C0350723C5F80035019BBA
:1097A000ABB13B68627943F307355201002DC3F337
:1097B0000733D2B21EDB164C661986F8002301224D
:1097C0006D0903F01F0302FA03F344F82530242344
:1097D00003FB081100234B7701230B7703B0BDE88F
:1097E000F08FC6F808B5AFE743F00403CFE743F0C6
:1097F0000603CCE7074C03F00F03E254E7E7082029
:10980000ECE71120EAE700BFD032002015960200F5
:1098100000E100E014ED00E070B50579224C24234E
:109820006B43E35893B103681A0B43F30733002BE0
:109830000CDB02F01F015B0901228A4020331B4927
:1098400041F82320BFF34F8FBFF36F8F24236B4367
:10985000E218E35800687BB1154BC0F80833537F1A
:1098600053B101234361D0F80431002BFBD02423F2
:1098700003FB054300225A77242303FB05430026FC
:1098800093F82030FF2B1FBF03F5E0734FF0A04289
:10989000022142F82310C0F80065FFF7B7F924232E
:1098A00003FB0544267770BDD032002000E100E0C4
:1098B000520108002DE9F3410779474E24237B43E9
:1098C0001446F2180D46517F8646002940F08180EB
:1098D000F35823B114F0140F04BF0123537795E814
:1098E0000F004FF0240C0CFB076C0CF10C0888E8FF
:1098F0000F009CF81F20FF2A08D09CF81E1001239F
:1099000093404FF0A042C1B1C2F80835296821B197
:1099100001F06043B3F1005F06D1AA6882B102F0A2
:109920006043B3F1005F0BD0242303FB07660023E1
:109930007377102002B0BDE8F081C2F80C35E5E77E
:10994000DEF800306868C3F84415C3F84805E968D4
:10995000C3F834250022C3F83815C3F81821D3F80A
:1099600018210192019A14F0010218BF0122C3F8D4
:10997000502514F0020218BF0122C3F84025220727
:109980005CBF01221A6124227A43B258B2B9D3F8DB
:109990001821002AFBD0242303FB0766F27FFF2A4D
:1099A00007D0B07F012393404FF0A04218B1C2F816
:1099B0000C350020BEE7C2F80835BBE714F0040000
:1099C0004FF0400202D0C3F80823F2E7C3F80423A3
:1099D000B0E71120AEE700BFD0320020032811D835
:1099E000012A0AD101290FD100F10E02D2B20D4B8A
:1099F00000EB40001A54002070470129F7D00229DB
:109A000004D049B1072070470022F8E7054B00EB6E
:109A1000400018444270EEE7024B00EB400018444F
:109A20008270E8E7F432002008B50122022100200C
:109A3000FFF7D4FF08B1072810D107220221012027
:109A4000FFF7CCFF08B1072808D100210A220846F9
:109A5000FFF7C4FF10B1072808BF002008BD0000B1
:109A60000388102B10B502D0112B1ED010BD1A4C3C
:109A70002168B1B901220846FFF7B0FF08B10728F5
:109A800024D1072202210120FFF7A8FF08B10728EF
:109A90001CD1042202210020FFF7A0FF08B10728F3
:109AA00014D1236801332360E0E70B4A1368013BBC
:109AB0001360002BDAD1FFF7B7FF0028D6D0074B91
:109AC0001B68002BD2D0BDE810401847034B1B6821
:109AD000002BE6D09847E4E7043300200033002051
:109AE0000B4B0222C3F8F0254FF400310022C3F8DB
:109AF000F425C3F818150121C3F81015C3F814256F
:109B0000C3F80023034AC3F82C26C3F83016704765
:109B10000070004048A80020074B0122C3F8002530
:109B20001A60D3F80021002AFBD00022C3F80021DC
:109B300001225A60704700BF0070004008B50B4B0F
:109B4000D3F8402182B1D3F80423D2030CD50022EC
:109B5000C3F84021FFF7E0FF054BD3F80421002AAA
:109B6000FBD00022C3F8042108BD00BF00A00040C4
:109B7000007000402DE9FF41174A18481368184D3E
:109B8000DFF86C80190442BF1B0C1B041360154BDB
:109B900012681549C01AC0080004C2F30B0240F055
:109BA00003000192FCF71CFF019A104902A801F082
:109BB000FEFD2E8802AF344602A801F069FE304453
:109BC000A04203D8288004B0BDE8F08117F8013B1B
:109BD00004F808300134EFE748A80020A4BF0200D1
:109BE00040A8002074BF020025C2020033C2020058
:109BF000083300200D4B0022C3F804250621012262
:109C0000DA60C3F810150A21C3F80825C3F8401517
:109C10004FF48031C3F804130549C02081F80A03CA
:109C20004FF4806008601A60704700BF00A00040D9
:109C300000E100E02DE9F3474FF400410020FCF77C
:109C400031FD08B1FDF7A6F86F4B704D7049ED1A64
:109C5000ED082D0445F003042046FCF7BDFE4FF04F
:109C6000A0430322C3F87427FFF73AFF00204FF404
:109C70000041FCF717FD08B1FDF78CF8FCF744FC38
:109C8000FFF7B8FF6348DFF80C82634F012100F053
:109C9000C1FC62492046FCF79FFE032698F800307D
:109CA000FBB95F4B5F485F69B84742685D484FF456
:109CB0008016B6FBF2F6B8475B490268B2FBF6F2D3
:109CC0002046FCF78DFE5949594F2046FCF784FE8B
:109CD00058495948012201F067FA3870F0B15749E4
:109CE0000DE039462046FCF777FE002000F070FBBF
:109CF000013E88F80000D1D10028D2D05049514D02
:109D00002046FCF769FE98F80030002B49D04E48F9
:109D100001F059FC002002B0BDE8F0874B49204615
:109D2000FCF75AFE4A494B4801F05AFC387060B9BA
:109D3000494EDFF8209106F1090A4749484601F0EB
:109D400082FC387018B14549D9E74549D7E7737A9D
:109D500045F005007BB94349FCF73EFE42492046E9
:109D6000FCF73AFE41493848332201F043FA387093
:109D7000A8B13F49C3E7337ADB0609D53D490190D5
:109D80005246FCF72DFE737A0198002BD5D1E2E7FD
:109D90003268394901905346FCF72BFEF3E7374907
:109DA000ADE72B68B3F5FA6F27D130492648204E2E
:109DB000332201F01FFA307020B12D492046FCF704
:109DC0000BFEA7E72E482F4D01F062FD2C490246FD
:109DD0002B461D4801F0EFFA307040B12A49204669
:109DE000FCF7FAFD184801F0EEFB2849E6E72A687F
:109DF00027492046FCF7F4FDF4E7FFF7BBFE2B688C
:109E000001332B607FE700BF74BF0200A4BF0200D4
:109E100037C202000C2B0020A8C302004CC2020073
:109E2000C8C10200E4C3020089C202009BC2020052
:109E300078A800204BC20200BCAA0020B0C20200D9
:109E40006BC2020044A800207CA80020C0C202000F
:109E5000DAC202004CA80020A4AA0020F8C2020026
:109E6000DCC2020049C202000FC302002CC3020080
:109E70004FC3020034C3020044C3020079C302008E
:109E8000083300203CA800209AC30200BEC3020091
:109E9000AAC30200082B00200369C26893429CBF3A
:109EA00080681B18013B981A70472DE9F843D0E9E8
:109EB00002940546A9EB04084068904520440F46EB
:109EC000144404D901F099FCEC60BDE8F8834246E3
:109ED000A4EB090401F091FC6868224607EB080135
:109EE000F0E72DE9F843C5680646894617464FF066
:109EF00000083469B3687068A54228BFE418013CC3
:109F0000621B5C1BBC4228BF3C46944228BF1446DF
:109F100049462844224601F070FCB3682544AB4210
:109F200008BF00253F1BA044A144F560E1D1404695
:109F3000BDE8F88310B5114C114AA2610223C4E9AF
:109F40000433104BE361A2644FF400730E4A0F49CF
:109F50002362E26400231022E01DA3626362E362D5
:109F6000A3656365E365226501F070FC084920463E
:109F700001F06CFC2023A37110BD00BF08AD0020D0
:109F800000C4020090AD002080AD002009C4020092
:109F90000DC4020070B5164B182400FB04451D4487
:109FA00004FB00331646DC6A012C0ED0022C18D0BC
:109FB000E4B92846FFF770FF864204D832462846A7
:109FC000FFF773FF3446204670BD2846FFF764FF55
:109FD0008642344628BF044622462846FFF765FFDE
:109FE000F1E72846BDE87040FFF77BBF0024EAE7B1
:109FF00008AD0020FFF79EBF034B1A8882420CBFBA
:10A0000018460020704700BFACAF0020024B9B6990
:10A0100003B11847704700BF90AF002037B50B461B
:10A02000497A0F4A79B9D2E901141D7A0246002D06
:10A0300018BF21465868FCF729FF78B103B0BDE886
:10A040003040FFF7E3BF00211972536933B1012299
:10A05000ADF806008DF8042001A8984703B030BD84
:10A0600090AF00204B8802889A4212D842889A42C8
:10A070000FD380888B8840F2F311884294BF021A74
:10A08000421A9A4205D80844984234BF0020012061
:10A0900070470020704700000388122B70B50146FE
:10A0A00059D004D8102B1ED0112B44D070BD502B8A
:10A0B000FCD12F4BC288DB899A42F7D1038A022B4D
:10A0C000F4D186883046FFF797FF05460028EDD08B
:10A0D00001F1120000F0F4F838BB6868FCF7EEFEFE
:10A0E0000028E3D009E0C37B012BDFD14FF6FF70DE
:10A0F000FFF782FF054620B90420BDE87040FFF756
:10A1000085BF1C4A8E880680002303721368C0F83E
:10A110000A305368C0F80E3010310A30FFF7A2FF42
:10A12000134B6872DB89002BC0D129463046BDE84D
:10A130007040FFF773BF8088FFF75EFF044600287A
:10A14000B4D04068FCF7BAFE08B1FFF75FFF4FF6E6
:10A15000FF732380AAE786883046FFF74DFF054648
:10A160000028A3D008310A30FFF77CFF6872DCE7D3
:10A1700090AF0020C0AF00200AB1FCF739BFFCF758
:10A1800040BF73B50191019C06466CB100252C4679
:10A19000294601A8FCF73FFF18B106EB4403013440
:10A1A0009D800135142DF3D13046346002B070BD6E
:10A1B0002DE9F04703888488103B8CB005460A2BB4
:10A1C00021D8DFE803F00640202020202020206551
:10A1D0004700DFF8E880D8F80830DB430093D8F870
:10A1E00004106846FCF743FF009901A8FFF7C9FF78
:10A1F0000DF108090027019B9F4207D3132C12D9A8
:10A200000420FCF7C7FD0CB0BDE8F08739F802ABBD
:10A2100000260136514608EB8600FCF7F2FE1E2EA2
:10A22000F7D10137E7E71F482146FCF7E1FE1E485A
:10A230002146FCF7DDFEEB7B022BE4D11B482146D7
:10A24000FCF7D6FEDFE7174821460CB0BDE8F04723
:10A25000FCF7D7BE027A16483F2A4FEA121521466C
:10A2600094BF00220122FFF787FF022D94BF002236
:10A27000012210482146FFF77FFF012D0E4894BFB1
:10A280000022012221460CB0BDE8F047FFF774BF61
:10A29000037A002BB7D1427A0548C2F3C0022146A7
:10A2A000F1E700BFD0AF0020CCAF0020D4AF00203A
:10A2B000E0AF0020DCAF0020D8AF0020C8AF002006
:10A2C000008800F001007047014B1878704700BF0C
:10A2D00044B0002007B508496846FDF7D4F9019B52
:10A2E00013B903B05DF804FBD3E90020904768463A
:10A2F000FDF7D3F9F3E700BF34C40200FFF7EABF6C
:10A3000061DF704730B5134DADF5017D4FF4FA7440
:10A310000DF1020103A8ADF80240FFF7F1FF70B99B
:10A32000294601A8FDF7AFF9029B002BF0D003A846
:10A33000D3E90021904701A8FDF7AFF9F4E705281C
:10A3400005D00DF5017DBDE83040FCF723BD0DF5CE
:10A35000017D30BD4CC40200024B1B780BB1FFF7EE
:10A36000D1BF704745B000204BDF70471FB50E4C82
:10A3700001A8FFF7F9FF70B9214602A8FDF783F99C
:10A38000039B002BF4D00198D3E90021904702A849
:10A39000FDF783F9F4E7052804D004B0BDE81040C8
:10A3A000FCF7F8BC04B010BD64C402000B78032BAA
:10A3B00009D8054B087A1B680C2200FB02334A7847
:10A3C0001A7200229A72704748B0002020BF70476E
:10A3D00038B5194B1B78834202462BD9174D00EB39
:10A3E000400329689C0001EB8303085910B3597A94
:10A3F000C90702D4587AC0B238BD596809B91049A2
:10A4000059600121997203680E491B68984720B171
:10A410002B682344EEE75B6898472B6823449A7ABD
:10A42000002AF8D11A7A002AF2D15A7A02F0FE02F2
:10A430005A72EDE70320DFE74CB0002048B000205F
:10A44000CDA30200ADA30200074B1B78834281BF5E
:10A45000064B1B6800EB400003EB800086BF407A90
:10A46000C0B20120704700BF4CB0002048B00020AF
:10A47000F0B515461C4A1278824285B02FD9002BC0
:10A480002DD01A4F00EB40003A68860002EB8000A6
:10A49000945934B3427AD20723D4CDE9015301232E
:10A4A00003918372236820465B69984703689D4245
:10A4B00002D3012005B0F0BD236801A99B682046A6
:10A4C00098470028F5D13B6833449A7A22B9187A24
:10A4D000003818BF0120EDE75B689847F3E70420D8
:10A4E000E8E70320E6E700BF4CB0002048B00020BA
:10A4F000F0B515461F4A1278824285B033D9002B39
:10A5000031D01D4F00EB40003A68860002EB80001E
:10A510009459002C29D0427AD20726D4427A520785
:10A5200025D4CDE90153012303918372236820468A
:10A530005B69984703689D4202D3012005B0F0BDD6
:10A54000236801A9DB68204698470028F5D13B68BD
:10A5500033449A7A22B9187A003818BF0120EDE7FF
:10A560005B689847F3E70420E8E70320E6E702206A
:10A57000E4E700BF4CB0002048B0002073B5234B87
:10A580001B7883420D46144639D901291CD0022973
:10A5900028D00123002934D100EB40001C4E8DF857
:10A5A000073084003368185903680DF107021B69EE
:10A5B0000021984708B1112803D19DF80730002BDE
:10A5C000F0D1284602B070BD114B00EB40001B6873
:10A5D00053F82000B8B103685B69984703682360AB
:10A5E0000025EEE70A4B00EB40001B6853F8200003
:10A5F00048B103685B69984743682380F0E7042506
:10A60000DFE71D46DDE70325DBE700BF4CB0002098
:10A6100048B00020024B1860024B1970704700BF11
:10A6200048B000204CB00020006870470B0A017051
:10A6300043700B0C090E8370C1707047024400F820
:10A64000011B9042FBD1704743690239023B8B42A8
:10A6500083BF4389806A01FB030000207047C2F377
:10A6600007238A76CB760378032B01BF120C0A7579
:10A67000120A4A757047026810B552B111460B466E
:10A6800011F8014B202C0CD93A2CF8D1511C8B42DB
:10A6900002D04FF0FF3005E01278302AF9D10133B3
:10A6A0000360002010BD38B50D46044618B90023DC
:10A6B00009202B6038BD0368002BF8D01A78002AD7
:10A6C000F5D0D98882889142F1D15878FFF7BCFE45
:10A6D00010F00100EBD12368EBE701380A4411F8D0
:10A6E000013B00F8013F9142F9D170472DE9F0415B
:10A6F000C66A00F1300804460123407832464146DC
:10A70000FFF7F6FE0546A8B9236AA269E070F31ABE
:10A71000934202D2A778012F02D82846BDE8F081E3
:10A72000A36960781E44324601234146FFF7E0FEEC
:10A73000013FF0E70125F0E7C3780BB1FFF7D6BF83
:10A740001846704738B5C36A8B4205460C4610D090
:10A75000FFF7F2FF60B922466878012305F1300166
:10A76000FFF786FE00281CBF4FF0FF340120EC628B
:10A7700038BD0020FCE70000002310B5C3704FF087
:10A78000FF33C3620446FFF7DDFF034618BBB4F88E
:10A790002E124AF6552291421FD194F83020E92A10
:10A7A00005D0226B0F4902F0FF128A4217D104F143
:10A7B0006600FFF739FF0C4A20F07F40904208D036
:10A7C00004F18200FFF730FF02F14C52904218BFB3
:10A7D0000223184610BD0423FBE70323F9E70223F5
:10A7E000F7E700BFEB009000464154002DE9FF4120
:10A7F00000230B600F461546FFF73DFF061EC0F213
:10A8000010818B4B53F82640002C00F00C813C60EB
:10A81000237805F0FE056BB16078FFF715FEC107E0
:10A8200008D41DB110F0040500D00A25284604B054
:10A83000BDE8F0810023F0B223706070FFF7C8FD1F
:10A84000C20700F1F2800DB14307EED4002120468B
:10A85000FFF792FF022840F0C8806F4604F5FB73B3
:10A8600004F236213A4613F8040C10B11846FFF7EB
:10A87000DBFE10338B4242F8040BF4D1002557F86D
:10A88000046B002E00F0A88031462046FFF774FFCD
:10A89000012800F2A280B4F83B30B3F5007F40F00D
:10A8A000A880B4F8461021B904F15400FFF7BCFEAB
:10A8B000014694F84030A1615A1E012AA37000F2AB
:10A8C000988094F83D506581002D00F092806A1EBA
:10A8D0002A4240F08E80B4F84180A4F8088018F035
:10A8E0000F0F40F08680B4F8430018B904F150000F
:10A8F000FFF79AFEE78F002F7BD001FB03FE07EBEB
:10A90000181CF444604574D3A0EB0C02AA42B2FBBD
:10A91000F5F36ED34FF6F57293426ED840F6F575A7
:10A92000AB428CBF02250125023337440CEB0602F3
:10A93000032D6361E6612762A26260D1B4F85A20F8
:10A9400052EA080255D104F15C00FFF76DFE9B004E
:10A95000606203F2FF13B1EB532F4AD34FF0FF3382
:10A96000C4E90333032D4FF0800323712BD1B4F8D6
:10A970006030012B27D1711C2046FFF7E3FE10BB8E
:10A98000B4F82E2220714AF655239A421BD104F1C5
:10A990003000FFF749FE274B984214D104F50570AB
:10A9A000FFF742FE03F1FF5303F5005320339842B3
:10A9B00009D104F50670FFF737FE206104F5077032
:10A9C000FFF732FEE0601C4A2570138801339BB20A
:10A9D0001380E380002529E703200135042D7FF44F
:10A9E0004EAF042805D1012520E70428FBD001281B
:10A9F00001D90D251AE700264DE7032594E7B8F1A4
:10AA0000000FF6D0022D4FEA430218BFD218774448
:10AA100018BF03F0010367620CBF134603EB520338
:10AA200097E70B2502E70C2500E70325FEE600BFAC
:10AA300050B000205252614154B0002001292DE94C
:10AA4000F04706460C46174673D943698B4270D9C6
:10AA50000378022B3FD0032B50D0012B69D101EB9F
:10AA60005108016A01EB5821FFF76CFE054638BB1F
:10AA700006F1300908F1010AC8F3080814F00104CE
:10AA80001FBF19F8083003F00F023B0103F0F00379
:10AA900014BF1343FBB209F80830316A0123F37085
:10AAA00001EB5A213046FFF74DFE054640B9CAF387
:10AAB000080A44B1C7F3071709F80A700123F370B5
:10AAC0002846BDE8F08719F80A30C7F3032723F0BA
:10AAD0000F031F43F0E7016A01EB1421FFF732FE79
:10AAE00005460028ECD1640006F1300304F4FF743D
:10AAF00018191F55C7F307274770DFE7016A01EBF5
:10AB0000D411FFF71FFE05460028D9D1A40006F195
:10AB1000300304F4FE741C442046FFF785FD27F043
:10AB2000704700F0704047EA00012046FFF77EFDC5
:10AB3000C4E70225C4E7F8B50446FFF7FDFD054666
:10AB4000002842D12378032B37D12779012F34D124
:10AB500004F1300601464FF4007230465523FFF7EA
:10AB60006DFD84F82E32AA2384F82F32522341221D
:10AB7000722184F8303084F83130612384F8323027
:10AB800084F8173284F8332084F8141284F81512EC
:10AB900084F81622216904F50670FFF747FDE16885
:10ABA00004F50770FFF742FDE26960780132E26266
:10ABB0003B463146FFF79CFC257100226078114628
:10ABC000FFF7DCFC003818BF0120F8BDF8B5002302
:10ABD0000246451E1C462E2615F8010F202804F1BA
:10ABE00001040AD0052808BFE520092C02BFCF18B0
:10ABF00001337E72CF18013378720B2CECD10B44E9
:10AC000000205872D37A0B7202F11C00FFF70CFD82
:10AC1000086002F11600FFF707FDC880000C88806D
:10AC2000F8BD03284B8B04BF8A8A43EA02431846C7
:10AC300070470129F8B506460C464ED9436999423A
:10AC40004BD20378022B29D0032B34D0012B44D1D3
:10AC500001EB5105016A01EB5521FFF773FD10B1BE
:10AC60004FF0FF30F8BD6F1C316AC5F3080535445D
:10AC700001EB5721304695F83050FFF763FD00286F
:10AC8000EED1C7F308073E44E30796F8300045EAE3
:10AC900000204CBF0009C0F30B00E3E7016A01EBA1
:10ACA0001421FFF74FFD0028DAD1640004F4FF748B
:10ACB0002644308ED6E7016A01EBD411FFF742FD3E
:10ACC0000028CDD1A40006F1300004F4FE74204425
:10ACD000FFF7AAFC20F07040C4E70120C2E737B5B7
:10ACE0000C46012C054611462BD943699C4228D2BB
:10ACF00022B14FF0FF32FFF7A1FE40B921462846AE
:10AD00000194FFF796FF0199044610B9002003B0A3
:10AD100030BD012815D0431C15D000222846FFF76E
:10AD20008DFE0028F3D1D5E90432911E8B4205D265
:10AD300001332B612B7943F001032B719442DDD356
:10AD4000E4E70220E3E70120E1E7F8B505460F4616
:10AD500071B9C668DEB143699E4228BF01263446F8
:10AD60006B6901349C4215D3012E12D8002405E0F2
:10AD7000FFF75FFF0128044602D801242046F8BDF2
:10AD8000431C2FD06B699842F8D33E46E7E7012673
:10AD9000E5E7022421462846FFF74BFF30B10128A2
:10ADA000EBD001301ED0A642DAD1DFE74FF0FF3200
:10ADB00021462846FFF742FE90B957B9D5E904323B
:10ADC000023A9342EC6010D32B7943F001032B71CC
:10ADD000D4E7224639462846FFF730FE0028EDD05A
:10ADE0000128CAD14FF0FF34C8E7013B2B61EBE7E4
:10ADF000826838B500230568036104469AB92B7848
:10AE0000022B01D96B6A6BB92B890BB9022038BDB3
:10AE10006B6AA361A3696261002BF7D03035E561ED
:10AE20000020F4E71A466B8963B911462068FFF7E2
:10AE300000FF431C02460BD00128E7D96B699842FA
:10AE4000F3D3E3E711462846FFF7FEFBA061E1E7F5
:10AE50000120DCE703692DE9F04703F1200883694D
:10AE600005468A4693B1B8F5001F0FD2C8F308090A
:10AE70000468B9F1000F4DD141690133836139B9DB
:10AE80002389B3EB581F45D80023AB6104200BE0A6
:10AE90006789013F17EA58273CD12046FFF7C9FED2
:10AEA0000128064602D80220BDE8F087421C01D1E5
:10AEB0000120F9E76369834226D8BAF1000FE3D095
:10AEC00069692868FFF741FF0646002835D0012848
:10AED000E9D0431CECD02046FFF72EFC01460028A9
:10AEE000E6D104F130004FF40072FFF7A7FB3146C2
:10AEF0002046FFF7A9FB4FF0010AE06263899F42F9
:10AF00000FD3E36ADB1BE3626E6131462046FFF735
:10AF10009BFBA86130344C44C5F81080EC610020E4
:10AF2000C2E784F803A02046FFF7E0FB0028BFD16A
:10AF3000E36A01330137E362E0E70720B4E700008A
:10AF40002DE9F041066880460C4611F8013B2F2B95
:10AF5000FAD05C2BF8D00023C8F8083023781F2BD8
:10AF600055D908F120050B2228462021FFF766FB62
:10AF7000002210460827235C202B00F1010108D98C
:10AF80002F2B01D05C2B4CD1605C2F2847D05C2844
:10AF900045D00C44002A5ED098F82020D8F80070E4
:10AFA000E52A04BF052288F82020212B34BF042382
:10AFB000002388F82B304046FFF71AFF002865D1A0
:10AFC000D8F818103846FFF7BDFB00285ED1D8F836
:10AFD0001C201378002B64D0D37A03F03F0388F849
:10AFE0000630D37A13F008000CD102F10B0C29467D
:10AFF00012F8013B11F801EB6245A3EB0E0343D0BD
:10B00000002BF5D000214046FFF724FFD6E7802330
:10B0100088F82B304046BDE8F041FFF7E9BE01312A
:10B02000B2E72E2B54D0974215D903F17F0C5FFA6B
:10B030008CFCBCF11E0F10D903F1200C5FFA8CFCC4
:10B04000BCF11C0F09D9DFF8A4C01CF8010B0028C3
:10B0500043D08342F9D1062021E014F801C0ACF1BD
:10B0600040013E2900F1020003D98CF080017C29C7
:10B07000F1D8791E8A42EED2511CAB5405F801C0BA
:10B0800002320146084676E7002BBBD198F82B30F8
:10B0900048B1042803D113F0040F08BF0520BDE810
:10B0A000F0810420F2E75A07F9D498F80630DB065D
:10B0B0000CD5D8F81010307806F13003C1F3080130
:10B0C0001944FFF7AEFDC8F808004CE70520E6E795
:10B0D0000B2FC0D008220B27D4E7A3F16100192859
:10B0E00001D8203BDBB2AB540132CBE770C4020085
:10B0F00038B5056804460420A16909B9A8B11CE067
:10B100002846FFF71FFBC0B9E3691A78C2B1DB7AA2
:10B11000E52A03F03F03A37109D02E2A07D00F2B95
:10B1200005D023F02003082B01D0002038BD0021DA
:10B130002046FFF78FFE0028DED00023A361F5E74D
:10B140000420FAE770B506680546FFF751FE04468D
:10B1500028BBA9693046FFF7F5FA0446F8B9EB6950
:10B160001B78E52B14D1A9693046FFF7EBFA0446AA
:10B1700060B901462022E869FFF760FAE8690B220E
:10B1800005F12001FFF7A9FA0123F370204670BDF5
:10B19000002BE8D001212846FFF75CFED7E7042CFE
:10B1A00008BF0724F2E700001FB5CDE9001003A88F
:10B1B00014460391FFF75FFA031E15DB0C4A52F8A1
:10B1C000231009B100200870019808B10021017016
:10B1D00042F8230030B1012C08D1002201A96846B1
:10B1E000FFF704FB04B010BD0B20FBE70020F9E7DC
:10B1F00050B000202DE9F0438FB01746019104466E
:10B20000002800F0D68002F03F052A4602A901A8D6
:10B21000FFF7ECFA0646002852D1029B01990393EE
:10B2200003A8FFF78DFE20B99DF93730002BB8BF7A
:10B23000062017F01C0F00F09C80002847D004283F
:10B240003ED103A8FFF77EFF002839D145F008055D
:10B250000A9BDDF808900027212148225A749F7329
:10B26000DF7319740A9B5A769F75DF7519760A9BEE
:10B270002022DA720A9999F80000FFF7D2FC3A46C8
:10B2800080464846FFF7EBF90A9B1F775F779F7769
:10B29000DF77029B0122DA70B8F1000F20D003980B
:10B2A000D3F82C903A464146FFF719FD40B9029871
:10B2B0004946FFF747FA029A08F1FF33D36078B1A5
:10B2C00000232360064630460FB0BDE8F0839DF8AA
:10B2D000123013F0110F56D1780764D43907B7D460
:10B2E000029F2907FB6A0A9923626162387848BF86
:10B2F00045F04005FFF795FCA06001F11C00FFF749
:10B3000093F90021FB88276004F12807E0604FF4DF
:10B310000072A38025746174E16161613846FFF7B2
:10B320008DF9AA06CFD5D4F80C80B8F1000FCAD099
:10B33000029BA1685D89C4F814806D02454524D341
:10B340000020A1610028BBD1C8F30803002BBAD0AC
:10B35000029D2846FFF778F948B300EB5822E261D6
:10B36000687801233946FFF783F80028ABD0012025
:10B37000A6E70028A4D19DF81230DA0615D4BF073D
:10B38000AED5D807ACD507209AE72068FFF751FC67
:10B3900001280146A8EB050803D9431CCED10120A2
:10B3A000CFE70220CDE708208AE7042088E70220C3
:10B3B00086E7092687E72DE9F04F994685B00023F7
:10B3C0008846C9F8003003A904461646FFF76BF912
:10B3D000054620BB657C15BB237C9A0740F1AA80FB
:10B3E0006369F34228BFDE4304F1280A9EB1636912
:10B3F000C3F30802002A40F08B80039A5789013F6B
:10B4000017EA53271ED173B9A06870B901462068A6
:10B41000FFF79BFC48B9237C43F040032374284684
:10B4200005B0BDE8F08FA169F1E7012802D102253E
:10B430006574F4E7431C01D10125F9E7A368A06115
:10B4400003B9A06094F91030002B0CDA0398E2697C
:10B45000407801235146FFF74BF80028ECD1237CBC
:10B4600003F07F032374DDF80CB0A1695846FFF7A1
:10B47000EBF80028DBD0B6F5007F07EB000235D3F0
:10B48000BBF80A1007EB562088424FEA56239BF878
:10B49000010088BFCB1B4146CDE90023FFF728F808
:10B4A0000028C9D1E169009A019B891A99420CD2FE
:10B4B0004FF4007208EB412150460093FFF70DF95D
:10B4C000227C009B02F07F0222745F026369E268C3
:10B4D0003B4463619A422CBFE260E360D9F80030DC
:10B4E0003B44B844C9F80030F61B7FE7E369934258
:10B4F0000DD0E1686369994209D99BF80100009277
:10B5000001235146FEF7B4FF009A002894D1E2616E
:10B510006069C0F30800C0F50077B74228BF37461E
:10B520003A4641465044FFF7D8F8237C63F07F0346
:10B530002374CBE7072572E773B501A90546FFF72A
:10B54000B2F80446002839D12B7C13F0400435D0E2
:10B550001B060CD50198EA694078012305F1280102
:10B56000FEF7C6FF68BB2B7C03F07F032B74296AB0
:10B570000198FFF7E7F8044600BB6E6AF37A43F0E0
:10B580002003F372AA6828683146FFF768F8E96873
:10B5900006F11C00FFF74AF8212333760198B475B1
:10B5A000482373760123F475B474F474C370FFF701
:10B5B000C2FA2B7C23F0400304462B74204602B0D1
:10B5C00070BD0124FAE713B50446FFF7B5FF28B9AB
:10B5D00001A92046FFF767F800B9206002B010BD4E
:10B5E0001FB50446019148B3002203A901A8FFF743
:10B5F000FDF870B9039B019923602046FFF7A0FC7A
:10B60000F0B994F92B30002B0CDBA379DB0603D4C3
:10B610000520002323600FE0039BE1691878FFF702
:10B6200000FBA060039BDB88A3802046FFF7E0FBC4
:10B630000428EDD00028ECD104B010BD0920FBE7B0
:10B640000428E5D0E5E737B50D4601A90446FFF724
:10B650002AF818B920461DB9FFF7CAFB03B030BD60
:10B66000FFF746FD10F0FB03F8D16B72A3691BB125
:10B67000E0692946FFF7AAFA00212046FFF7EAFB16
:10B68000042808BF0020E9E77F2805D8034B185C91
:10B69000034B5B5C18407047002070478CC402006D
:10B6A0000CC50200A0F16103192B98BF2038704728
:10B6B000A0F14103192B98BF203070477F2805D88F
:10B6C000034B185C034B5B5C1840704700207047CD
:10B6D0008CC402000CC50200A0F16103192B98BFB5
:10B6E00020387047A0F14103192B98BF20307047D4
:10B6F0007F299ABF017001206FF02E0070475AB168
:10B700000A787F2A0AD800B10260002119605960C6
:10B71000501A18BF01207047002070476FF02E00AC
:10B72000704710B504460846A2684AB123686168AC
:10B7300003F1010C8C4508BF00208B4208D2D05485
:10B74000E3682BB121686268914201D22146984793
:10B7500023680133236010BD70B54C1E09D4164612
:10B76000C5B229463046FFF7DCFF013CB4F1FF3F8C
:10B77000F7D170BD10F0100F08D108B510F4007F9C
:10B7800014BF30202020FFF7E7FF08BD70470000FE
:10B7900008B5034B5B689B681B68984708BD00BFF2
:10B7A000182B002008B50921FFF7F2FF08BD0EB4E1
:10B7B00000B586B007AA52F8041B05920390002337
:10B7C00004936FF00043029301A800F091F806B0D3
:10B7D0005DF804EB03B07047037853B159B10144ED
:10B7E000034613F8012F12B18B42FAD10B46181AF7
:10B7F00070470346FBE70346F9E7844640EA010346
:10B8000013F0030F18D18446202A0BD32DE9F0073B
:10B81000B1E8F807A0E8F807A2F12002202AF7D241
:10B82000BDE8F007042A07D351F8043B40F8043B75
:10B83000A2F10402042AF7D2002A05D011F8013B34
:10B8400000F8013B013AF9D160467047024610F01A
:10B85000030F16D111F0030F13D12DE9F0004FF0B3
:10B8600001374FF0803351F8044BA4EB070525EA6C
:10B8700004051D4002D142F8044BF4E7A1F1040194
:10B88000F0BC11F8013B02F8013B002BF9D17047E5
:10B8900000F1010110F0030F11D010F8012B002A64
:10B8A00023D010F0030F0AD010F8012B002A1CD06F
:10B8B00010F0030F03D010F8012B002A15D02DE94A
:10B8C00070004FF001324FF0803350F8044BA4EB7E
:10B8D000020525EA04051D4000D1F6E7A0F10400A9
:10B8E00070BC10F8012B002AFBD1A0EB01007047BF
:10B8F0002DE9F04F89B007460392002303600C4600
:10B9000014F8011B002900F0FC82DFF818B5EBE207
:10B91000002507E05E2868D145F4805501E045F038
:10B9200040051C46234613F8010B3028F2D81F2887
:10B9300037D9A0F12002102A33D801A151F822F002
:10B940001FB90200A3B90200A3B9020085B9020021
:10B95000A3B90200A3B90200A3B902008BB9020087
:10B96000A3B90200A3B90200A3B9020091B9020071
:10B97000A3B9020097B90200A3B90200A3B902005B
:10B980009DB9020045F08005CBE745F40045C8E7C6
:10B9900045F02005C5E745F01005C2E745F4007500
:10B9A000BFE72A2821D1039A111D0391D2F800A0E4
:10B9B000BAF1000FBCBFCAF1000A45F010051878B3
:10B9C000A31C2AEAEA7A2E2826D00021742847D020
:10B9D0007A2845D06C2800F0A8804C2800F0AB8075
:10B9E000682800F0B8801C463DE0A0F13002D2B2D9
:10B9F000092A88BF4FF0000AE3D84FF0000A0AEB8B
:10BA00008A0A303800EB4A0A13F8010BA0F1300221
:10BA1000D2B2092AF3D9D4E718782A280AD1039A8E
:10BA2000111D03911168587802330029CEDB45F4CB
:10BA30008075CBE70133A0F13002D2B2092A88BF6A
:10BA40000021F4D8002101EB8101303800EB4101E5
:10BA500013F8010BA0F13002D2B2092AF3D9E4E7BE
:10BA60001C4614F8010B002800F05782A0F12503B2
:10BA7000DBB2532B62D8A0F12503532B5ED8DFE84D
:10BA800013F076005D005D005D005D005D005D000F
:10BA90005D005D005D005D005D005D005D005D00BE
:10BAA0005D005D005D005D005D005D005D005D00AE
:10BAB0005D005D005D005D005D005D005D005D009E
:10BAC0005D005D005D005D005D005D005D005D008E
:10BAD0005D005D005D005D005D005D005D005D007E
:10BAE0005D005D005D005D00EC005D005D005D00DF
:10BAF0005D005D005D005D005D005D005D007B0040
:10BB000021015D005D005D005D0021015D005D00C3
:10BB10005D005D0095000F01D2005D005D00A60094
:10BB20005D001A015D005D00EE001C4614F8010B7B
:10BB300045F0010597E745F001051C46B54B1E6829
:10BB4000002E00F0CE8103AB0193009153462A46AC
:10BB50003946B047C5E11878682803D05C1C45F029
:10BB6000040580E745F008059C1C58787BE72521F3
:10BB70003846FFF7D6FDB4E1039B1A1D03921E78E9
:10BB80000AF1FF3A3A4651462846FFF7F3FD31469F
:10BB90003846FFF7C6FDA94619F0100F00F0A18145
:10BBA0003A4651462020FFF7D7FD9AE115F0080FDD
:10BBB00006D03A68039B191D03911B681A7090E127
:10BBC000039B1A1D03921B683A681A6089E1039B64
:10BBD0001A1D0392D3F800808F4BB8F1000F08BFF5
:10BBE0009846464625F4007915F4807F16D04046E5
:10BBF000FFF7F2FD0546AAEB050A3A4651464846CC
:10BC0000FFF7B8FD002DC7D016F8011B3846FFF727
:10BC100088FDA8EB0603EB42F6D1BDE74046FFF7EF
:10BC200037FE0546E7E7039B1A1D03921B6815F0D4
:10BC3000800F0CBF0026232645F4807508211A4684
:10BC4000002B00F02A8105AB4FF0000805F4005CE2
:10BC5000A64660468C460146D2E045F4005515F0F4
:10BC6000800F1BD043F2780643F25803782818BFA0
:10BC70001E4615F4807F01D025F4007515F4804F21
:10BC800032D0039B1A1D03921B6815F0040F1FD0BE
:10BC90001BB2002B20DA5B422D262DE00026E8E7C0
:10BCA00015F0800F0CBF0026302615F4807FE5D0FC
:10BCB00025F40075E2E715F4807F07D025F40075C0
:10BCC0000026DBE745F480450026D7E70026D5E7C8
:10BCD00015F0080FDDD0DBB215F0200F61D115F0A3
:10BCE000400F18BF202607E0039B1A1D03921B6814
:10BCF00015F0040F50D09BB215F4807F14BF25F4CB
:10BD0000007501215838202800F2AF8001A252F8B6
:10BD100020F000BF3FBC02006BBE02006BBE020001
:10BD20006BBE02006BBE02006BBE02006BBE020067
:10BD30006BBE02006BBE02006BBE02006BBE020057
:10BD40006BBE0200CFBD02006BBE02006BBE0200E4
:10BD50006BBE02006BBE0200CFBD02006BBE0200D4
:10BD60006BBE02006BBE02006BBE02006BBE020027
:10BD7000A7BD02003FBC02006BBE02006BBE02000A
:10BD80006BBE02006BBE0200CFBD02006BBE0200A4
:10BD90006BBE02003FBC020015F0080FACD0DBB256
:10BDA000AAE72B26A8E71A464FF00008002B5ED022
:10BDB00005A84FF0000803F00703303300F8013BFB
:10BDC00008F10108D2081346002AF4D14FE01846C2
:10BDD0004FF00008002B4AD04FF0000805F4004E49
:10BDE0004FF02C0973468E4619462FE002F00F00E3
:10BDF0000A4C205C03F8010B08F10108120906D077
:10BE00000029F3D002F00F00054C205CF2E77446E5
:10BE100061462CE058B00020E0C60200C0C6020017
:10BE2000D0C60200CDCCCCCC08AB03EB080CABFBEE
:10BE30000032D20802EB8203A0EB430330330CF84C
:10BE40000C3C08F1010809280DD910460029EBD057
:10BE500008F00303032BE7D108AB434403F80C9C21
:10BE600008F10108E0E7714601E04FF00008A1EB9E
:10BE7000080121EAE179AAEB090AAAEB080AFF2ED8
:10BE80000ED9AAF1020AC6F307213846FFF749FC8A
:10BE9000F1B23846FFF745FC04E04FF00008E6E752
:10BEA000002E3DD13A4651462846FFF763FC3A46FC
:10BEB00049463020FFF750FCB8F1000F0EDD0DF1C0
:10BEC000140908F1FF38C84498F80010464638466F
:10BED000FFF727FCC14508F1FF38F5D115F0100F29
:10BEE00009D114F8011B61B125293FF411AD384681
:10BEF000FFF717FCF5E73A4651462020FFF72CFCE8
:10BF0000EFE7BB682BB13A6879688A423CBF0021F1
:10BF10009954386809B0BDE8F08F4FF0FF30F9E769
:08BF20000AF1FF3AB4E700BF8B
:08BF28009187020000000000F7
:10BF3000B1A1020000000000619A020000000000B0
:08BF400099A0020000000000BE
:08BF48002D880200000000003A
:10BF500059A30200000000006DA3020000000000D1
:10BF6000702B0020382C0020402C0020782B002043
:04BF700018000000B5
:10BF7400F2C1020000000000F8C10200000000004D
:10BF8400FFC102000000000020C202000000000007
:10BF940003C202000000000008C20200000000000A
:10BFA40066C002000000030368C102000000000034
:10BFB4008CC102000000000021C402000000000047
:10BFC400ECC102000000000014C4020000000303DE
:10BFD40029C402000000030340C40200000003035C
:10BFE40058C4020000000303A6C1020000000000C0
:08BFF400AFC1020000000000D3
:10BFFC0028C002000000000045C00200D82A002022
:10C00C005CC102000000000034C00200E02A0020E5
:10C01C00000000000338FDD870470000D563020013
:10C02C0041640200D1630200756172745F6C6F67CA
:10C03C005F6261636B656E64007274745F6C6F67D2
:10C04C005F6261636B656E64004261636B656E6415
:10C05C007320666C75736865640061707000000015
:10C06C00603000207F000000E03000201B5B313B83
:10C07C0033316D0025734C6F67732064726F707071
:10C08C006564202825642925730D0A001B5B306D1F
:10C09C00002573003C25733E2025733A2000202593
:10C0AC0030327800202020007C002563001B5B319F
:10C0BC003B33306D001B5B313B33326D001B5B310E
:10C0CC003B33336D001B5B313B33346D001B5B31F9
:10C0DC003B33356D001B5B313B33366D001B5B31E5
:10C0EC003B33376D007761726E696E6700696E66FF
:10C0FC006F0064656275670098C00200B9C00200E9
:10C10C0078C00200C1C00200C9C00200D1C0020048
:10C11C00D9C00200E1C00200E9C00200000000002A
:10C12C0079C10200F1C00200F9C00200FEC0020099
:10C13C00FFFFFFFFFFFFFFFFFFFFFFFFFFFFFFFF03
:10C14C0000000000000000000000D6010601000005
:10C15C00C16C0200656D0200BD6C02006170705F05
:10C16C00627574746F6E00466174616C20657272D6
:10C17C006F720053797374656D207265736574000A
:10C18C006170705F74696D657200303132333435B3
:10C19C00363738394142434445467077725F6D6794
:10C1AC006D7400736F72746C69737400000000001E
:10C1BC000030004000000000010000006583020018
:10C1CC00118302009982020021820200F181020097
:10C1DC000F820200000001010000000101000000BC
:10C1EC00636C6F636B00434C4F434B004750494F9C
:10C1FC00544500505253005541525400554152542D
:10C20C0045000000FFFFFFFF0006FF00000000409C
:10C21C00000000005350494D004144432056616CCE
:10C22C0075653A2025640025640A000D0A464154C0
:10C23C004653206578616D706C652E0D0A0D0A00F1
:10C24C00496E697469616C697A696E672064697397
:10C25C006B20302028534443292E2E2E0D0A0044E7
:10C26C0069736B20696E697469616C697A61746950
:10C27C006F6E206661696C65642E0D0A00436170F7
:10C28C0061636974793A202564204D420D0A004D92
:10C29C006F756E74696E6720766F6C756D652E2E7A
:10C2AC002E0D0A004D6F756E74206661696C6564A5
:10C2BC002E0D0A000D0A204C697374696E67206498
:10C2CC0069726563746F72793A202F0D0A002F0022
:10C2DC004469726563746F7279206C697374696EEA
:10C2EC0067206661696C6564210D0A00446972659A
:10C2FC0063746F72792072656164206661696C6524
:10C30C00642E0057726974696E6720746F206669B9
:10C31C006C65204455382E5458542E2E2E0D0A0080
:10C32C004455382E545854002020203C4449523E49
:10C33C0020202025730D0A00253931752020257306
:10C34C000D0A00556E61626C6520746F206F70650C
:10C35C006E206F72206372656174652066696C650E
:10C36C003A204455382E5458542E0D0A00537563F8
:10C37C006365737366756C6C206F70656E2066698F
:10C38C006C65203A204455382E5458542E00577260
:10C39C00697465206661696C65640D0A2E002564FC
:10C3AC00206279746573207772697474656E2E0DD2
:10C3BC000A00636C6F73652066696C652074686134
:10C3CC006E6820636F6E67004E6F72646963005312
:10C3DC00444300312E303000C8C10200D4C30200E7
:10C3EC00DBC30200DFC30200000200000B131A1CA7
:10C3FC00ECAC00205465726D696E616C0052545443
:10C40C0000534547474552006E72665F626C655F2C
:10C41C006761747400626C655F6E7573006E726632
:10C42C005F7364680000000050BF020060BF020030
:10C43C00080000006E72665F7364685F626C650072
:10C44C0030BF020048BF0200080000006E72665F39
:10C45C007364685F736F630028BF020030BF020013
:10C46C0008000000222A2B2C3A3B3C3D3E3F5B5DF2
:10C47C007C7F000043000000504F534958000000DF
:10C48C002020202020202020206828282828202038
:10C49C002020202020202020202020202020202090
:10C4AC004810101010101010101010101010101048
:10C4BC0084848484848484848484101010101010E8
:10C4CC001081818181818101010101010101010141
:10C4DC0001010101010101010101011010101010F5
:10C4EC001082828282828202020202020202020212
:10C4FC0002020202020202020202021010101020BA
:10C50C0000070320041702010857104080000000A8
:10C51C0080C4020084C5020098C6020053756E00E8
:10C52C004D6F6E0054756500576564005468750056
:10C53C004672690053617400000000004A616E008D
:10C54C00466562004D617200417072004D61790068
:10C55C004A756E004A756C00417567005365700032
:10C56C004F6374004E6F760044656300000000005A
:10C57C00414D00504D000000BCC60200B8C6020080
:10C58C00B8C60200B8C60200B8C60200B8C602009F
:10C59C00B8C60200B8C60200B8C60200B8C602008F
:10C5AC00FFFFFFFFFFFFFFFFFFFFFFFFFFFF00008D
:10C5BC00F8C5020028C5020034C6020048C50200B6
:10C5CC007CC50200DCC502008CC60200E8C5020076
:10C5DC00256D2F25642F257900000000256120256D
:10C5EC0062202565202554202559000053756E6462
:10C5FC006179004D6F6E6461790054756573646187
:10C60C0079005765646E657364617900546875725E
:10C61C007364617900467269646179005361747561
:10C62C0072646179000000004A616E756172790074
:10C63C004665627275617279004D61726368004182
:10C64C007072696C004D6179004A756E65004A75AF
:10C65C006C79004175677573740053657074656D02
:10C66C00626572004F63746F626572004E6F76651F
:10C67C006D62657200446563656D626572000000F1
:10C68C0025483A254D3A25530000000089B6020092
:10C69C00A5B60200B1B60200BDB60200D9B60200C2
:10C6AC00E5B60200F1B60200FFB602000000000081
:10C6BC002E00000030313233343536373839616270
:10C6CC00636465663031323334353637383941423C
:0BC6DC0043444546286E756C6C290035
:10C6E80000000000FF00000000000000FF00000044
:10C6F8000000000000200040000000000020004072
:10C708000000000000100140110004000090D00358
:10C7180001000000E4C30200000000000001000066
:10C728001CC502001CC502001CC502001CC5020075
:04C738001CC502001A
:040000032000637501
:00000001FF
